:10000000A0EF32F00000000091EF2EF000000000A1
:10001000000000000000000010EF31F00B6A0A6AD7
:10002000096A00500402F4CF09F0F3CF08F0015040
:100030000502F4CF0BF0F3CF0AF000500502F350A5
:100040000926F4500A22E86A0B2201500402F350F8
:100050000926F4500A22E86A0B2208C000F009C001
:1000600001F00AC002F00BC003F012001E0E716E08
:10007000100E0001E66F040EE76FE6C0E1FFE7C077
:10008000E2FFE69EE6C0E1FFE7C0E2FFE69C040E69
:10009000E625E16E000EE721E26EE68C180E4D6E4D
:1000A000040E4E6E4DC0E1FF4EC0E2FFE69E4DC015
:1000B000E1FF4EC0E2FFE69C040E4D24E16E000E0F
:1000C0004E20E26EE68C020EE625E16E000EE72180
:1000D000E26ED2C0E6FFD3C0E6FF010EE625E16E78
:1000E000000EE721E26E400EE66EE6C0E9FFE7C0D3
:1000F000EAFFEECF00F0E6C0E1FFE7C0E2FF400E0E
:100100000014E66EE6C0E9FFE7C0EAFFEECF00F0BC
:10011000E6C0E1FFE7C0E2FF880E0010E66EE6C031
:10012000CEF0E7C0CFF0040EE619006E00C0E6F096
:1001300012000AAE029E000E1200C7B409D01F0EB4
:10014000C514016E0150000A03E1010E006E01D0DA
:10015000006A12000B840BAEB5EF00F0010E036EC7
:10016000026A016A006A0A360232FF0E1200026A4F
:10017000016A006A086A036A000E12000B820BAE65
:10018000C8EF00F003680268016800680A360232AE
:10019000FF0E1200000E545C02E1080E535C11E2E7
:1001A00053C003F054C004F00001CC51000A03E135
:1001B000010ECC6F05D0CC51010A02E1020ECC6FCA
:1001C00004D0080E036E000E046E00014BC0E1FF68
:1001D0004CC0E2FFE6924BC0E1FF4CC0E2FFE6906C
:1001E0004BC0E9FF4CC0EAFFEECF00F04BC0E1FF8F
:1001F0004CC0E2FF04500010E66E010E4B24E16E8D
:10020000000E4C20E26E03C0E6FF0350535C006E0C
:1002100004505458016E00C053F001C054F0280E31
:10022000CA6F040ECB6F52B02FD0035004102BE0D6
:100230004FC0F6FF50C0F7FF51C0F8FF0900F5CFDF
:1002400000F0CAC0E1FFCBC0E2FF00C0E6FFCA4B2E
:10025000CB2B010E4F24006E000E5020016E000EBD
:100260005120026E00C04FF001C050F002C051F0AA
:10027000010E035C006E000E0458016E00C003F016
:1002800001C004F0D2D724D00350041021E04FC0A5
:10029000E9FF50C0EAFFCAC0E1FFCBC0E2FFEECFEA
:1002A000E6FFCA4BCB2B010E4F24006E000E5020F0
:1002B000016E00C04FF001C050F0010E035C006EF3
:1002C000000E0458016E00C003F001C004F0DCD73A
:1002D000120004012051800AD8A473D0C00E526EBF
:1002E00065D09B0E006E640E016E000E026E00C0A3
:1002F0004FF001C050F002C051F0120E536E000ECC
:10030000546E5FD0030E006E000E016E22C404F026
:10031000000E056E83DE5E0E0024E96E000E0120E5
:10032000EA6EEECF4FF0EECF50F0EECF51F0020E6E
:100330004F24F66E000E5020F76E000E5120F86E1E
:100340000900F5CF00F00900F5CF01F000C053F02F
:1003500001C054F036D022510001E35D23E3030EC7
:10036000006E000E016E22C404F0000E056E56DE13
:10037000790E0024E96E000E0120EA6EEECF4FF0F8
:10038000EECF50F0EECF51F04FC0F6FF50C0F7FF68
:1003900051C0F8FF0900F5CF00F000C053F0000E87
:1003A000546E01D0526A0DD0526A0BD00401235111
:1003B000010A97E02351020AA5E02351030ACBE08A
:1003C000F3D71200528E716A0001D46B22C43DF043
:1003D0003D50000A03E1100ECD6F03D0200ECD6F0B
:1003E00045DE120020C401F01F0E01160150010A63
:1003F00001E08DD004012451000A01E088D0215190
:10040000060A3FE134D03D50010A17E1500E006E5C
:10041000630E016E000E026E120E0026000E012207
:10042000022200C04FF001C050F002C051F0090E8E
:10043000536E000E546EC00E526E23D03D50010A12
:1004400012E1E70E006E630E016E000E026E00C038
:100450004FF001C050F002C051F0210E536E000E5B
:10046000546EC00E526E0DD0800E526E0AD0040132
:100470002351210AC8E02351220AE0E02351230A34
:10048000F3E020C401F0600E0116050E006E00506E
:1004900004E00132019EFF0FFBD70150010A01E089
:1004A00036D022D034D033D0550E4F6E000E506E61
:1004B000010E536E000E546EC10E526E28D0800E87
:1004C000526E23C455F023D0560E4F6E000E506E60
:1004D000010E536E000E546E810E526E18D0800EB7
:1004E000526E22C456F013D004012151010ADAE001
:1004F0002151090AD8E02151020AD6E021510A0A05
:10050000DEE02151030AE0E021510B0AE8E012008D
:100510000401286B296B47D00401528E2881000109
:10052000E051010A02E10401288352D0528E50D0DA
:100530000401528E24BF16D024C403F00F0E0316FC
:1005400003C000F0000E016E003600900136E40E8C
:100550000024E96E000E0120EA6EEECF04F0EECF2B
:1005600005F015D024C403F00F0E031603C000F0ED
:10057000000E016E0036009001364B0E0024E96E2D
:10058000000E0120EA6EEECF04F0EECF05F004C0BD
:10059000E9FF05C0EAFFEECF01F001A403D004019A
:1005A000010E286F15D020C401F01F0E0116015056
:1005B000000AB2E020C401F01F0E01160150010A2A
:1005C000B5E020C401F01F0E01160150020AB0E090
:1005D00052AE07D0280E4F6E040E506E5280020E9F
:1005E000536E120004012251010A11E120C401F0EE
:1005F0001F0E01160150000A0AE1528E2151030A12
:1006000004E1010E0001E06F02D00001E06B040183
:100610002251000AD8A48BD020C401F01F0E01166D
:100620000150020AD8A483D024C401F00F0E011691
:100630000150000AD8B47BD0528E24BF16D024C4F7
:1006400003F00F0E031603C000F0000E016E00361B
:1006500000900136E40E0024E96E000E0120EA6EDF
:10066000EECF04F0EECF05F015D024C403F00F0E4A
:10067000031603C000F0000E016E00360090013634
:100680004B0E0024E96E000E0120EA6EEECF04F05E
:10069000EECF05F02151030A07E104C0E1FF05C0D8
:1006A000E2FF840EE66E43D024C400F00F0E001665
:1006B000700E026E0F0E036E00500226D8B0032A91
:1006C00002C0E9FF03C0EAFFFE0EEE14006EEECF9B
:1006D00001F0FF0E011602C0E1FF03C0E2FF00C0FF
:1006E000E6FF01C0E6FF24AF11D004C0E1FF05C062
:1006F000E2FFE66A040E0418006E00C004F004C0B5
:10070000E1FF05C0E2FF400EE66E11D004C0E1FF3C
:1007100005C0E2FF880EE66E040E0418006E00C0ED
:1007200004F004C0E1FF05C0E2FFC80EE66E12004F
:100730000101306B316B3151120802E130518E08EA
:1007400008E3FBDC005201E004D00101304B312B07
:10075000F2D70101120E315D02E18F0E305D03E32D
:100760007B0E006E05D0C580C5A001D0FDD7006A04
:1007700012000CB0FBEF03F00CA2A2EF04F00E6A23
:10078000000E026412EF04F0F00E0214D8A4DDEFA4
:1007900003F0023A01380F0B02260138F00B016E0C
:1007A00000380F0B01260038F00B006E08380F0BD5
:1007B00000260838F00B086E0E84D89002BEF6EFC3
:1007C00003F008360036013602360E2A02BEF6EF76
:1007D00003F008360036013602360E2A02BEF6EF66
:1007E00003F008360036013602360E2A0E50036436
:1007F00097EF04F0035E0BBC08AE9CEF04F0D880CA
:10080000800E08640030000E002201220222D8A0CF
:100810009CEF04F0023201320032034AA2EF04F0EE
:100820009CEF04F001C002F000C001F008C000F02D
:10083000086A000E0E86026449EF04F0F00E0214FE
:10084000D8A431EF04F0023A01380F0B0226013828
:10085000F00B016E00380F0B01260038F00B006E14
:100860000E84D89002BEF6EF03F000360136023651
:100870000E2A02BEF6EF03F00036013602360E2ACB
:1008800002BEF6EF03F00036013602360E2AF6EF0E
:1008900003F001C002F000C001F0006A000E0E96E5
:1008A0000E88026476EF04F0F00E0214D8A461EF13
:1008B00004F0023A01380F0B02260138F00B016EEA
:1008C0000E84D89002BEF6EF03F0013602360E2AEF
:1008D00002BEF6EF03F0013602360E2A02BEF6EF34
:1008E00003F0013602360E2AF6EF03F001C002F0E3
:1008F000016A000E0E860264A7EF04F0F00E0214E7
:10090000D8A485EF04F0023A0E84D89002BEF6EF28
:1009100003F002360E2A02BEF6EF03F002360E2A6C
:1009200002BEF6EF03F002360E2AF6EF03F0010ED8
:100930000C6E10DCAAEF04F0020E0C6E99EC00F0C5
:10094000AAEF04F0040E0C6E19DCAAEF04F0080EF6
:100950000C6E0DDC120020C401F0600E0116050EB5
:10096000006E005004E00132019EFF0FFBD70150E2
:10097000000A01E05AD036D0528E080E0001CD6F29
:1009800054D0A7DC52D01EDD50D03D0E4F6E000E6D
:10099000506E5280010E536E528E47D0B9DD45D055
:1009A00021DE43D0D40E006E000E016E04012451EE
:1009B0000026D8B0012A00C04FF001C050F052808C
:1009C000010E536E528E31D0528ED40EE16E000E57
:1009D000E26E2451E126D8B0E22A22C4E6FF25D0F7
:1009E00024D023D004012151050AC6E02151060A72
:1009F000C8E02151090AC7E02151080AC6E0215187
:100A0000000ACCE02151010ACBE02151030AC8E0E1
:100A100021510A0AC7E021510B0AD6E02151070AE9
:100A2000DFE021510C0ADDE0DCD71200160E6F6EFC
:100A30009F0E6B6E3B0E696E12006D9852BE4BD0CE
:100A400043AE29D0020E4A6E010E4B24E16E000E19
:100A50004C20E26EE66A4BC0E1FF4CC0E2FFC80EDC
:100A6000E66E010E0001C825E16E000EC921E26E9E
:100A7000080EE66E020EC825E16E000EC921E26E78
:100A8000280EE66E040EE66EC8C0E1FFC9C0E2FFA4
:100A9000C80EE66E1FD00001010EC825E16E000EE3
:100AA000C921E26E080EE66E020EC825E16E000E48
:100AB000C921E26E200EE66E040EE66EC8C0E1FFAC
:100AC000C9C0E2FF8C0EE66E4BC0E1FF4CC0E2FFF6
:100AD000840EE66E80D043BE7ED0040120AF53D09A
:100AE0005450275D02E15350265D04E226C453F0C2
:100AF00027C454F0CAEC00F0010E4A6E010E00014A
:100B0000C825E16E000EC921E26E080EE66E020EE7
:100B1000C825E16E000EC921E26E200EE66E040EBD
:100B2000E66EC8C0E1FFC9C0E2FF800EE66EDF6B73
:100B3000010ED925E16E000EDA21E26E080EE66E96
:100B4000020ED925E16E000EDA21E26E200EE66E6D
:100B5000040EE66ED9C0E1FFDAC0E2FF840EE66E55
:100B6000010EDF6F020E4B24E16E000E4C20E26E90
:100B7000280EE66E040EE66E4BC0E1FF4CC0E2FFAD
:100B8000C80EE66E28D00001020E4A6E010E4B24FC
:100B9000E16E000E4C20E26EE66A4BC0E1FF4CC0F5
:100BA000E2FFC80EE66E010EC825E16E000EC921F7
:100BB000E26E080EE66E020EC825E16E000EC92137
:100BC000E26E280EE66E040EE66EC8C0E1FFC9C0F4
:100BD000E2FFC80EE66E1200C5841200500E5E6E73
:100BE000630E5F6E000E0001606FFA0E796F640E87
:100BF0007A6F000E7B6FC50E7C6F630E7D6F000EEB
:100C00007E6FF00E7F6F620E806F000E816F12009C
:100C10000001D55302E0F2EC01F01200010E0001D8
:100C2000D925E96E000EDA21EA6EEECF00F000C0A1
:100C300002F0000E455C02E10250445C03E244C055
:100C400002F00AD00250445C006E000E4558016E5E
:100C500000C044F001C045F0036A0250035C1CE28E
:100C6000280EE96E040EEA6E0350E926D8B0EA2A8F
:100C7000EECF00F041C0E1FF42C0E2FF00C0E6FF5E
:100C8000010E4124006E000E4220016E00C041F0B2
:100C900001C042F0032AE1D7000E006E4550005C0F
:100CA00002E14450000828E2010EC825E16E000E62
:100CB000C921E26E080EE66E020EC825E16E000E36
:100CC000C921E26E280EE66E040EE66ED9C0E9FF79
:100CD000DAC0EAFFEECF00F000BC07D0C8C0E1FFE9
:100CE000C9C0E2FFC80EE66E06D0C8C0E1FFC9C0A9
:100CF000E2FF880EE66E19D0010EC825E16E000EE7
:100D0000C921E26E080EE66E020EC825E16E000EE5
:100D1000C921E26E200EE66E040EE66EC8C0E1FF49
:100D2000C9C0E2FF840EE66E439E12009E9630C15B
:100D3000C9FFC7A401D0FDD79EB601D0FDD7C5BC61
:100D400002D0006A03D0C584020E006E12004A6A07
:100D50004BC0E1FF4CC0E2FFE66A040E4B18E16EA7
:100D60004CC0E2FF000EE21AE66A43BE439E120048
:100D7000DFDC2DC130F1DADF00C02FF12EC130F100
:100D8000D5DF00C02FF128DF2FC100F01200A19A9B
:100D90001200086A080E0C6E003408360450085E13
:100DA000D8B002D00826D89000360C2EF5D7120005
:100DB0000B800BAEE4EF06F0026A0AAEFF0E026E85
:100DC000016E006E0A360232FF0E1200040E4B183E
:100DD000006E00C04BF00001CD51080A0AE122C4A8
:100DE0006EFF6E50000803E2100ECD6F02D0040EAD
:100DF000CD6F4A50010A3CE1020E4B24E16E000E19
:100E00004C20E26E280EE66E040EE66ECAEC00F090
:100E10000001CC51020A07E14BC0E1FF4CC0E2FFE8
:100E2000840EE66E24D0040E4B18006E00C04BF00A
:100E30004BC0E9FF4CC0EAFFEECF00F000BC0CD085
:100E4000040E4B18006E00C04BF04BC0E1FF4CC0CD
:100E5000E2FFC80EE66E0BD0040E4B18006E00C009
:100E60004BF04BC0E1FF4CC0E2FF880EE66E01D0B4
:100E70006EDF12006D92699468A403D0FB0E6816B1
:100E8000FBD71200025006180E6E086A096A0B6A38
:100E90000350076435EF08F006500A6E068E028E86
:100EA00003500B6E0750036E000E0B6485EF07F0C6
:100EB0000B50075ED8B426EF08F0070E0764F4EF76
:100EC00007F0075E00C008F001C000F002C001F0AA
:100ED000026A074E26EF08F00764C9EF07F0075EC5
:100EE00000C008F001C000F0016A074E26EF08F0CC
:100EF0000764A7EF07F0075E00C008F0006A074E1E
:100F000026EF08F007648EEF07F00AC002F005C074
:100F100001F004C000F0086A52EF09F0030E076404
:100F200099EF07F0075E08380F0B086E074E26EFA3
:100F300008F0D8900832074E26EF08F0D890083213
:100F4000074E26EF08F0D890083226EF08F0030E7F
:100F50000764B8EF07F0075E08380F0B086E00381B
:100F6000F00B082600380F0B006E074E26EF08F036
:100F7000D89000320832074E26EF08F0D8900032A1
:100F80000832074E26EF08F0D8900032083226EFDC
:100F900008F0030E0764E0EF07F0075E08380F0B58
:100FA000086E0038F00B082600380F0B006E013871
:100FB000F00B002601380F0B016E074E26EF08F0EC
:100FC000D890013200320832074E26EF08F0D89050
:100FD000013200320832074E26EF08F0D890013275
:100FE0000032083226EF08F0030E076411EF08F014
:100FF000075E08380F0B086E0038F00B0826003823
:101000000F0B006E0138F00B002601380F0B016E3C
:101010000238F00B012602380F0B026E074E26EF46
:1010200008F0D8900232013200320832074E26EF23
:1010300008F0D8900232013200320832074E26EF13
:1010400008F0D8900232013200320832096A000EEC
:101050000EAE1AEF09F0081E001E011E021E082A1D
:101060000022012202221AEF09F00750D8A43BEF18
:1010700008F052EF09F0096A02C00AF0028E068EEB
:101080000750035C076ED8B40DEF09F0070E076434
:10109000DBEF08F0075E0450096E0550046E065041
:1010A000056E066A074E0DEF09F0070E0764B0EFF4
:1010B00008F0075E0450096E0550046E056A074E7D
:1010C0000DEF09F0070E07648EEF08F0075E04507D
:1010D000096E046A074E0DEF09F0070E076475EFFD
:1010E00008F00AC002F052EF09F0030E076480EF27
:1010F00008F0075E09380F0B096E074E0DEF09F077
:10110000D8900932074E0DEF09F0D8900932074EFA
:101110000DEF09F0D89009320DEF09F0030E0764C6
:101120009FEF08F0075E09380F0B096E0438F00BCB
:10113000092604380F0B046E074E0DEF09F0D89006
:1011400004320932074E0DEF09F0D890043209320B
:10115000074E0DEF09F0D890043209320DEF09F077
:10116000030E0764C7EF08F0075E09380F0B096E1E
:101170000438F00B092604380F0B046E0538F00B09
:10118000042605380F0B056E074E0DEF09F0D890B9
:10119000053204320932074E0DEF09F0D8900532BE
:1011A00004320932074E0DEF09F0D89005320432AF
:1011B00009320DEF09F0030E0764F8EF08F0075E3F
:1011C00009380F0B096E0438F00B092604380F0B91
:1011D000046E0538F00B042605380F0B056E063833
:1011E000F00B052606380F0B066E074E0DEF09F0C3
:1011F000D8900632053204320932074E0DEF09F05D
:10120000D8900632053204320932074E0DEF09F04C
:10121000D8900632053204320932086A000E0EAE4A
:101220001AEF09F0091E041E051E061E092A0422D3
:1012300005220622095008260450002205500122EA
:10124000065002220EBE31EF09F0D8A040EF09F09F
:101250000232013200320832033E40EF09F04CEF17
:1012600009F0D8B046EF09F0000E081E001E011E5E
:10127000021E082A0022012202220A7E46EF09F0FD
:10128000010E0C6EB9EC03F054EF09F0020E0C6E77
:10129000B9EC03F054EF09F0040E0C6EBEEC00F054
:1012A00054EF09F0000E0C6E1200086A096A000E75
:1012B00007620364DAEF09F0025006180A6E07505D
:1012C00003267E0ED8A06BEF09F0035ED8B0DFEFE7
:1012D00009F06FEF09F0035ED8A0E4EF09F0028E89
:1012E000068E02C00EF001C00BF000C00DF00050E1
:1012F0000402F4CF0CF001500502F4CF00F0F3CF5C
:1013000008F00402F3500C26F4500822000E0022CC
:101310000D500502F3500C26F4500822000E002256
:1013200002500402F3500826F45000220250050235
:10133000016A000E0122F3500026F45001220D50E4
:101340000602F3500826F4500022026A000E012221
:1013500002220B500602F3500026F4500122000E28
:1013600002220E500602F3500126F450022202BE61
:10137000C2EF09F008360036013602360306D8B44B
:10138000E4EF09F0D5EF09F0D880800E0864003052
:10139000000E002201220222D8A0D5EF09F002326D
:1013A00001320032034ADFEF09F00AAE029E000E5E
:1013B000E7EF09F0010EB7EC00F0E7EF09F0020EDD
:1013C000BEEC00F0E7EF09F0040EAAEC00F012000A
:1013D00005DCCE6BCF6BE16BE26B6A6A686A16EC78
:1013E00005F06D8C6E6A716A6D9CD06BD16B000ECE
:1013F000D15D02E1080ED05D17E2D0C000F0D1C08F
:1014000001F0003600900136003600900136000EE3
:101410000024E16E040E0120E26EE66AE66AE66AE6
:10142000E66AD04BD12BE3D7160E706E68A603D0B8
:10143000F70E6816FBD7526A436A446A456A6D988C
:10144000080E4B6E040E4C6E3D6ACD6B120070A000
:1014500019D0D9C0E9FFDAC0EAFFEECF01F00150A0
:10146000800A0FE14BC0E9FF4CC0EAFFEECF01F06C
:101470000150840A06E1D9C0E1FFDAC0E2FF8C0E18
:10148000E66E7090DF0E681612006984EF0E681623
:101490006D8212004A50020A03E10EEC06F01FD0E2
:1014A00056DC0001DF51000A19E1010EC825E16E8A
:1014B000000EC921E26E080EE66E020EC825E16E2E
:1014C000000EC921E26E200EE66E040EE66EC8C064
:1014D000E1FFC9C0E2FF8C0EE66E01D0DF6B1200A7
:1014E0000134083609360450085E0550D8A0053C82
:1014F000095E003601360F0E0C6E013408360936CF
:10150000045000A006D0085E0550D8A0053C095E36
:1015100005D008260550D8B0053C0926003601360E
:101520000C2EEBD700B006D0045008260550D8B0DA
:10153000053C0926000012000B6A0B86FF0E120004
:101540004BC0E9FF4CC0EAFFEECF00F000AE05D083
:101550004BC0E1FF4CC0E2FFE66A0001CC6B4A6A77
:10156000536A546A526AABEC04F008EC06F01DECC6
:1015700005F012000D6A086A0050D8B4000C041877
:101580000A6E0ABE0D1E0B6A04AE02D0041E042AA7
:1015900000AE02D0001E002A005004100A6E0ABEDF
:1015A0001FD00450085E0036003408360450082668
:1015B0000036060E0C6E00340836045000B0085E8B
:1015C00000A0082600360C2EF6D700A008260BB087
:1015D00015D00DAE000C001E002A081E082A000CB3
:1015E00004AE09D000BE04D00050086E006AF1D7E6
:1015F000006A002A000C001E0B2AD3D7082A0450C8
:10160000085CD8A4E6D7086A002A00AEE2D7FF0C2F
:1016100012000B6A0C6A0A6A086A0350D8B491EF88
:101620000BF0028E9E0E035E03BE1CEF0BF0D8B4CF
:101630001CEF0BF081EF0BF0036C080E035CD8A0DD
:101640004EEF0BF0036E083600C008F001C000F04A
:1016500002C001F0026A080E035CD8A04EEF0BF046
:10166000036E083600C008F001C000F0016A080EE1
:10167000035CD8A04EEF0BF0036E083600C008F0F4
:10168000006A080E035CD8A04EEF0BF0036E08361C
:10169000086A0350D8A4D8905AEF0BF00350D8B47E
:1016A0005AEF0BF0D8900232013200320832032E8A
:1016B00052EF0BF00BBC08A06BEF0BF0D8A06BEF58
:1016C0000BF0082AD8B4002AD8B4012AD8B4022AC8
:1016D00002BE95EF0BF00AAE91EF0BF0021E011E59
:1016E000001E081E082AD8B4002AD8B4012AD8B48B
:1016F000022A91EF0BF0026A016A006A086A91EF10
:101700000BF00B800BAE9BEF0BF0026A0AAE9BEF67
:101710000BF0026E016E006E086E0A3602329BEF0D
:101720000BF0000E0C6A9CEF0BF0010E0C6ED8EC67
:1017300006F09CEF0BF0FF0E0250036E0150026E9C
:101740000050016E0850006E120001012851000A7D
:1017500012E027C100F0000E016E00360090013645
:101760004B0E0024E96E000E0120EA6EEECF04F06D
:10177000EECF05F011D027C100F0000E016E00364B
:1017800000900136E40E0024E96E000E0120EA6E9E
:10179000EECF04F0EECF05F0020E0424E16E000E51
:1017A0000520E26E29C1E6FF2AC1E6FF010E0424EE
:1017B000E16E000E0520E26E2BC1E6FF04C0E9FFDA
:1017C00005C0EAFFEECF00F004C0E1FF05C0E2FF74
:1017D000400E0014E66E04C0E9FF05C0EAFFEECF3C
:1017E00000F004C0E1FF05C0E2FF880E0010E66EC5
:1017F0002851000A1BE027C100F0000E016E0036E0
:10180000009001364B0E0024026E000E0120036E84
:1018100002C0E9FF03C0EAFF040EEE18006E02C02A
:10182000E1FF03C0E2FF00C0E6FF1AD027C100F0CD
:10183000000E016E003600900136E40E0024026EA8
:10184000000E0120036E02C0E9FF03C0EAFF040E90
:10185000EE18006E02C0E1FF03C0E2FF00C0E6FF29
:1018600004C000F005C001F012000001CD51000AD3
:101870000BE16D6A696A16EC05F06DB602D06D86F3
:10188000FCD70001010ECD6FCD51010A08E16DBA00
:1018900006D0686A696A69806988020ECD6F68A49B
:1018A00006D069A404D0FB0E68163AEC07F06DA2CE
:1018B00003D0C7EC06F0DCD068A018D069A016D021
:1018C00087DD040ECD6F200E0401026F040E036F3E
:1018D000080E016F000E0015006E00C000F48C0EA3
:1018E0000011006E00C000F4FE0E681668A805D056
:1018F00069A803D0CADDEF0E681668AC04D069ACE5
:1019000002D0BF0E681668AA03D069AA01D09FDD75
:1019100068A202D069B26A6A040E0001CD5D03E2DA
:10192000C7EC06F0A5D069A6A1D00101286B040E72
:10193000285DD8B09BD068A695D06CCFD8F0F70EB4
:101940006816780E0001D815016E0150000AD8A45F
:1019500088D0FD0ED815016E026AFF0E0216000E29
:10196000021802E1000E01186CE17E0ED815016E1E
:1019700001C003F00332039E03C000F0000E016EAD
:10198000003600900136003600900136000E00242B
:10199000026E040E0120036E02C0D9F003C0DAF01B
:1019A00002C0C8F003C0C9F0040EC819006E00C020
:1019B000C8F002C0E9FF03C0EAFFEECF00F000C0AC
:1019C00001F03C0E01160132019E0132019E0150D0
:1019D0000D0A35E1020ED925E96E000EDA21EA6E14
:1019E000EECF01F0EECF02F00250040A02E1280E21
:1019F000011823E1020ED925E16E000EDA21E26E14
:101A0000200EE66E040EE66E0101276B080E275DC0
:101A100014E2200EE16E040EE26E2751E126D8B0EA
:101A2000E22A280EE96E040EEA6E2751E926D8B0A4
:101A3000EA2AEECFE6FF272BE9D782DD01D02ADDA7
:101A40000FD00001FD0ED815016E026AFF0E0216BE
:101A5000000E021802E1040E011802E1E6EC06F0A5
:101A600000D001D003D00101282B61D7C7EC06F0CC
:101A700012000B6A0C6A086A0350D8B4BDEF0DF06F
:101A800002C00AF0028E9E0E035E03AEADEF0DF0B3
:101A9000036C080E035CD8A07AEF0DF0036E0836D5
:101AA00000C008F001C000F002C001F0026A080E98
:101AB000035CD8A07AEF0DF0036E083600C008F082
:101AC00001C000F0016A080E035CD8A07AEF0DF0A7
:101AD000036E083600C008F0006A080E035CD8A048
:101AE0007AEF0DF0036E0836086A0350D8A4D89038
:101AF00086EF0DF00350D8B486EF0DF0D890023287
:101B0000013200320832032E7EEF0DF00BBC08A02C
:101B100097EF0DF0D8A097EF0DF0082AD8B4002A5F
:101B2000D8B4012AD8B4022A02BEC1EF0DF00AAE21
:101B3000BDEF0DF0021E011E001E081E082AD8B4BB
:101B4000002AD8B4012AD8B4022ABDEF0DF0026AE7
:101B5000016A006A086ABDEF0DF00B800BAEC8EF9A
:101B60000DF0026A0AAEC8EF0DF0026E016E006E53
:101B7000086E0A360232C8EF0DF00C6A000EC9EF8B
:101B80000DF0010E0C6E000ED8EC06F0C9EF0DF052
:101B9000FF0E0250036E0150026E0050016E08509D
:101BA000006E1200000E0101281902E1000E271933
:101BB00002E1016A0AD027C1E9FF28C1EAFFEECF9E
:101BC00000F0000E00BE010E016E01C000F0120018
:101BD0006E0E0101275DD8A0CAD0640E046E27C125
:101BE00000F0C9EC06F0120E0024056E066A000E25
:101BF000062205C000F006C001F0000E06BEFF0E72
:101C0000026E036E0036009001360236033600364F
:101C10000090013602360336BC0E0024F66E620ECA
:101C20000120F76E000E0220F86E0900F5CF00F0DB
:101C30000900F5CF01F00900F5CF02F00900F5CF5A
:101C400003F0000E046E000E056E000E066E7E0E92
:101C5000076E55EC09F000C028F101C029F102C05F
:101C60002AF103C02BF1640E046E27C100F0C9EC09
:101C700006F008C000F00A0E046EC9EC06F0090E6A
:101C80000024056E066A000E062205C000F006C09C
:101C900001F0000E06BEFF0E026E036E00360090CD
:101CA000013602360336003600900136023603361E
:101CB000BC0E0024F66E620E0120F76E000E0220AC
:101CC000F86E0900F5CF00F00900F5CF01F009002A
:101CD000F5CF02F00900F5CF03F028C104F029C1C7
:101CE00005F02AC106F02BC107F055EC09F000C041
:101CF00028F101C029F102C02AF103C02BF10A0E1C
:101D0000046E27C100F0C9EC06F008C000F000C066
:101D100001F0000E026E036E046E01360190023671
:101D20000336043601360190023603360436BC0E03
:101D30000124F66E620E0220F76E000E0320F86E8C
:101D40000900F5CF00F00900F5CF01F00900F5CF4B
:101D500002F00900F5CF03F028C104F029C105F015
:101D60002AC106F02BC107F055EC09F0B1D027517C
:101D70000A08D8B07ED00A0E046E27C100F0C9EC64
:101D800006F0090E0024056E066A000E062205C044
:101D900000F006C001F0000E06BEFF0E026E036EDC
:101DA00000360090013602360336003600900136C8
:101DB00002360336BC0E0024F66E620E0120F76E6A
:101DC000000E0220F86E0900F5CF00F00900F5CFF3
:101DD00001F00900F5CF02F00900F5CF03F0000E85
:101DE000046E000E056E000E066E7E0E076E55EC3C
:101DF00009F000C028F101C029F102C02AF103C096
:101E00002BF10A0E046E27C100F0C9EC06F008C0E1
:101E100000F000C001F0000E026E036E046E013689
:101E2000019002360336043601360190023603363D
:101E30000436BC0E0124F66E620E0220F76E000E10
:101E40000320F86E0900F5CF00F00900F5CF01F08E
:101E50000900F5CF02F00900F5CF03F028C104F026
:101E600029C105F02AC106F02BC107F055EC09F095
:101E70002FD027C100F0000E016E026E036E0036F7
:101E800000900136023603360036009001360236E5
:101E90000336BC0E0024F66E620E0120F76E000EB3
:101EA0000220F86E0900F5CF00F00900F5CF01F02F
:101EB0000900F5CF02F00900F5CF03F0000E046E23
:101EC000000E056E000E066E7E0E076E55EC09F0D4
:101ED0001200F00E01012715006E0086008000C080
:101EE00028F13EC02DF1040E00102E6FB8EC06F064
:101EF00000C03FF0000E406E130E0D6E0D2EFED78B
:101F0000000000003EC02DF1FB0E010128152E6FD0
:101F1000B8EC06F000C03FF0000E406E130E0D6EE0
:101F20000D2EFED70000000027C100F00036009003
:101F3000003600900036009000360090F00E00163B
:101F40000086008000C028F13EC02DF1040E001074
:101F500001012E6FB8EC06F000C03FF0000E406E9D
:101F6000130E0D6E0D2EFED7000000003EC02DF1A9
:101F7000FB0E010128152E6FB8EC06F000C03FF0F3
:101F8000000E406E130E0D6E0D2EFED700000000E9
:101F900012000050086E0150006E0250016E035096
:101FA000026E036A0B6A0C6A9E0E036E0A6A020EC8
:101FB0000C6EB9EC03F012000B6A0A6A096A086A2F
:101FC0000E6A033408360450085E0550D8A0053C5C
:101FD000095E0650D8A0063C0A5E0750D8A0073C10
:101FE0000B5EE86AD8A0010E0E5E0336070E0C6E7B
:101FF0000334083609360A360B360E36045003A071
:1020000012D0085E0550D8A0053C095E0650D8A045
:10201000063C0A5E0750D8A0073C0B5EE86AD8A0D1
:10202000010E0E5E11D008260550D8B0053C0926D9
:102030000650D8B0063C0A260750D8B0073C0B26FD
:10204000E86AD8B0010E0E2603360C2ED1D7023422
:10205000083609360A360B360E36045003A012D065
:10206000085E0550D8A0053C095E0650D8A0063C85
:102070000A5E0750D8A0073C0B5EE86AD8A0010EA4
:102080000E5E11D008260550D8B0053C0926065032
:10209000D8B0063C0A260750D8B0073C0B26E86AA1
:1020A000D8B0010E0E260236070E0C6E023408362A
:1020B00009360A360B360E36045002A012D0085EDE
:1020C0000550D8A0053C095E0650D8A0063C0A5E23
:1020D0000750D8A0073C0B5EE86AD8A0010E0E5E40
:1020E00011D008260550D8B0053C09260650D8B0B6
:1020F000063C0A260750D8B0073C0B26E86AD8B041
:10210000010E0E2602360C2ED1D7013408360936C0
:102110000A360B360E36045002A012D0085E055067
:10212000D8A0053C095E0650D8A0063C0A5E0750C0
:10213000D8A0073C0B5EE86AD8A0010E0E5E11D055
:1021400008260550D8B0053C09260650D8B0063CF4
:102150000A260750D8B0073C0B26E86AD8B0010E13
:102160000E260136070E0C6E0134083609360A3683
:102170000B360E36045001A012D0085E0550D8A0D0
:10218000053C095E0650D8A0063C0A5E0750D8A060
:10219000073C0B5EE86AD8A0010E0E5E11D008263F
:1021A0000550D8B0053C09260650D8B0063C0A2692
:1021B0000750D8B0073C0B26E86AD8B0010E0E26AF
:1021C00001360C2ED1D70034083609360A360B36C4
:1021D0000E36045001A012D0085E0550D8A0053C70
:1021E000095E0650D8A0063C0A5E0750D8A0073CFE
:1021F0000B5EE86AD8A0010E0E5E11D008260550CD
:10220000D8B0053C09260650D8B0063C0A2607502F
:10221000D8B0073C0B26E86AD8B0010E0E2600366F
:10222000070E0C6E0034083609360A360B360E36A9
:10223000045000A012D0085E0550D8A0053C095EED
:102240000650D8A0063C0A5E0750D8A0073C0B5E9B
:10225000E86AD8A0010E0E5E11D008260550D8B04D
:10226000053C09260650D8B0063C0A260750D8B0CF
:10227000073C0B26E86AD8B0010E0E2600360C2E5D
:10228000D1D700B00ED0045008260550D8B0053C78
:1022900009260650D8B0063C0A260750D8B0073C9D
:1022A0000B2612009B0E006E640E016E000E026E75
:1022B0000E0E0024F66E000E0120F76E000E0220B6
:1022C000F86E0900F5CF03F003C004F00F0E0024F0
:1022D000F66E000E0120F76E000E0220F86E090067
:1022E000F5CF01F00150035C12E29B0E006E640E0C
:1022F000016E000E026E0F0E0024F66E000E01201D
:10230000F76E000E0220F86E0900F5CF04F09B0E68
:10231000006E640E016E000E026E100E0024F66E4A
:10232000000E0120F76E000E0220F86E0900F5CFB6
:1023300001F00150045C12E29B0E006E640E016E0F
:10234000000E026E100E0024F66E000E0120F76ED5
:10235000000E0220F86E0900F5CF04F004C000F072
:1023600012000C6A0E6A0250D8A4CAEF11F001C024
:1023700002F000C001F0006A0E860250D8A4CAEF35
:1023800011F001C002F0016A0E960E880250D8B416
:10239000DCEF11F00E50035ED8A4D8A0E2EF11F0EC
:1023A000D89002BEE8EF11F0003601360236032E57
:1023B000D1EF11F0E2EF11F0010E0C6EB7EC00F06E
:1023C000ECEF11F0020E0C6EAAEC00F0ECEF11F045
:1023D000040E0C6E99EC00F01200067E42EC07F041
:1023E000120001012751390806E3300E275D03E38F
:1023F000010E006E01D0006A1200D08EA28AA08A5F
:10240000F28E12000450000A12E10550000A0FE19A
:102410000650000A0CE10750000A09E1FF0E006EA9
:10242000FF0E016E7F0E026EFF0E036EA8D0086ACB
:10243000096A0750D8B4ADEF12F00350D8B4B2EF28
:1024400012F0025006180A6E028E068E0E6A02C044
:1024500008F001C00CF000C00DF004500D5E0550F6
:10246000D8A0053C0C5E0650D8A0063C085E086A61
:102470000C6A0D6AD8A044EF12F0D89002320132F3
:1024800000320832010E0E6E0750035ED8A051EFE5
:1024900012F07E0E0E240326D8B0B7EF12F057EFDD
:1024A00012F07E0E0E240326D8A0BCEF12F0180EF8
:1024B0000B6E0D360C3608360036013602360E36F7
:1024C0000450005E0550D8A0053C015E0650D8A01F
:1024D000063C025E06340E120EA072EF12F00D8062
:1024E0007DEF12F0045000260550D8B0053C0126BF
:1024F0000650D8B0062802260D900B2E59EF12F088
:10250000A3EF12F0D8900036013602360E36045092
:10251000005E0550D8A0053C015E0650D8A0063CE0
:10252000025E06340E10010B0D26D8B00C2AD8B46A
:10253000082AD8A4A3EF12F008320C320D32032A75
:10254000D8B4B7EF12F00AAE089E0850026E0C50D5
:10255000016E0D50006EBFEF12F0010E9CEC0AF000
:10256000BFEF12F0020EB7EC00F0BFEF12F0040E56
:10257000BEEC00F0BFEF12F0080EAAEC00F0120063
:10258000800E01012719006E800E000A005CD8B091
:102590006DD127510008016E01C027F1800E01188E
:1025A000006E800E6E0A005CD8A0C0D0640E046E6F
:1025B00027C100F0BAEC0AF0120E0024056E000EDE
:1025C00000BEFF0E066E000E062205C000F006C01B
:1025D00001F0000E06BEFF0E026E036E0036009084
:1025E00001360236033600360090013602360336D5
:1025F000BC0E0024F66E620E0120F76E000E022063
:10260000F86E0900F5CF28F10900F5CF29F109008E
:10261000F5CF2AF10900F5CF2BF1640E046E27C126
:1026200000F0BAEC0AF008C000F00A0E046EBAEC32
:102630000AF0090E0024056E000E00BEFF0E066EA5
:10264000000E062205C000F006C001F0000E06BE16
:10265000FF0E026E036E003600900136023603361E
:1026600000360090013602360336BC0E0024F66EAA
:10267000620E0120F76E000E0220F86E0900F5CF01
:1026800000F00900F5CF01F00900F5CF02F00900D4
:10269000F5CF03F028C104F029C105F02AC106F0E6
:1026A0002BC107F055EC09F000C028F101C029F159
:1026B00002C02AF103C02BF10A0E046E27C100F0FC
:1026C000BAEC0AF008C000F000C001F0000E00BE35
:1026D000FF0E026E036E046E013601900236033661
:1026E000043601360190023603360436BC0E01244E
:1026F000F66E620E0220F76E000E0320F86E0900DF
:10270000F5CF00F00900F5CF01F00900F5CF02F098
:102710000900F5CF03F028C104F029C105F02AC152
:1027200006F02BC107F055EC09F007D2800E0A0A1B
:10273000006E800E2719005C71E20A0E046E27C13C
:1027400000F0BAEC0AF0090E0024056E000E00BE7F
:10275000FF0E066E000E062205C000F006C001F056
:10276000000E06BEFF0E026E036E003600900136AC
:102770000236033600360090013602360336BC0EB0
:102780000024F66E620E0120F76E000E0220F86E35
:102790000900F5CF28F10900F5CF29F10900F5CF9F
:1027A0002AF10900F5CF2BF10A0E046E27C100F0C3
:1027B000BAEC0AF008C000F000C001F0000E00BE44
:1027C000FF0E026E036E046E013601900236033670
:1027D000043601360190023603360436BC0E01245D
:1027E000F66E620E0220F76E000E0320F86E0900EE
:1027F000F5CF00F00900F5CF01F00900F5CF02F0A8
:102800000900F5CF03F028C104F029C105F02AC161
:1028100006F02BC107F055EC09F08FD127C100F06D
:10282000000E27BFFF0E016E026E036E0036009091
:102830000136023603360036009001360236033682
:10284000BC0E0024F66E620E0120F76E000E022010
:10285000F86E0900F5CF00F00900F5CF01F009008E
:10286000F5CF02F00900F5CF03F067D1800E2719EC
:10287000006E800E6E0A005CD8A0C0D0640E046E9C
:1028800027C100F0BAEC0AF0120E0024056E000E0B
:1028900000BEFF0E066E000E062205C000F006C048
:1028A00001F0000E06BEFF0E026E036E00360090B1
:1028B0000136023603360036009001360236033602
:1028C000880E0024F66E620E0120F76E000E0220C4
:1028D000F86E0900F5CF28F10900F5CF29F10900BC
:1028E000F5CF2AF10900F5CF2BF1640E046E27C154
:1028F00000F0BAEC0AF008C000F00A0E046EBAEC60
:102900000AF0090E0024056E000E00BEFF0E066ED2
:10291000000E062205C000F006C001F0000E06BE43
:10292000FF0E026E036E003600900136023603364B
:1029300000360090013602360336880E0024F66E0B
:10294000620E0120F76E000E0220F86E0900F5CF2E
:1029500000F00900F5CF01F00900F5CF02F0090001
:10296000F5CF03F028C104F029C105F02AC106F013
:102970002BC107F055EC09F000C028F101C029F186
:1029800002C02AF103C02BF10A0E046E27C100F029
:10299000BAEC0AF008C000F000C001F0000E00BE62
:1029A000FF0E026E036E046E01360190023603368E
:1029B000043601360190023603360436880E0124AF
:1029C000F66E620E0220F76E000E0320F86E09000C
:1029D000F5CF00F00900F5CF01F00900F5CF02F0C6
:1029E0000900F5CF03F028C104F029C105F02AC180
:1029F00006F02BC107F055EC09F09FD0800E0A0AB3
:102A0000006E800E2719005C71E20A0E046E27C169
:102A100000F0BAEC0AF0090E0024056E000E00BEAC
:102A2000FF0E066E000E062205C000F006C001F083
:102A3000000E06BEFF0E026E036E003600900136D9
:102A40000236033600360090013602360336880E11
:102A50000024F66E620E0120F76E000E0220F86E62
:102A60000900F5CF28F10900F5CF29F10900F5CFCC
:102A70002AF10900F5CF2BF10A0E046E27C100F0F0
:102A8000BAEC0AF008C000F000C001F0000E00BE71
:102A9000FF0E026E036E046E01360190023603369D
:102AA000043601360190023603360436880E0124BE
:102AB000F66E620E0220F76E000E0320F86E09001B
:102AC000F5CF00F00900F5CF01F00900F5CF02F0D5
:102AD0000900F5CF03F028C104F029C105F02AC18F
:102AE00006F02BC107F055EC09F027D027C100F004
:102AF000000E27BFFF0E016E026E036E00360090BF
:102B000001360236033600360090013602360336AF
:102B1000880E0024F66E620E0120F76E000E022071
:102B2000F86E0900F5CF00F00900F5CF01F00900BB
:102B3000F5CF02F00900F5CF03F0120001012A6B76
:102B40002B6B2C6B020E2725F66E000E2821F76EDC
:102B5000000E2921F86E0900F5CF05F0030E272598
:102B6000F66E000E2821F76E000E2921F86E09007E
:102B7000F5CF00F000C003F0000E046E03C001F0BA
:102B8000006A05500024066E000E0120076E27C162
:102B900008F028C109F029C10AF0010E0824F66ED8
:102BA000000E0920F76E000E0A20F86E0900F5CF1E
:102BB00001F00150020A1BE1060E0824F66E000E19
:102BC0000920F76E000E0A20F86E0900F5CF01F01B
:102BD00001502A5D0CE2060E0824F66E000E092054
:102BE000F76E000E0A20F86E0900F5CF2AF1010EEB
:102BF0000824F66E000E0920F76E000E0A20F86E0B
:102C00000900F5CF01F00150040A1BE1080E082469
:102C1000F66E000E0920F76E000E0A20F86E09000D
:102C2000F5CF01F001502A5D0CE2080E0824F66E83
:102C3000000E0920F76E000E0A20F86E0900F5CF8D
:102C40002AF108C0F6FF09C0F7FF0AC0F8FF090023
:102C5000F5CF00F000502B25016E000E2C21026EE6
:102C600001C02BF102C02CF10750025C02E10650BA
:102C7000015C01E30FD008C0F6FF09C0F7FF0AC0EE
:102C8000F8FF0900F5CF00F000500826000E0922D9
:102C90000A2283D72AC100F012000A6A0350D8A47E
:102CA0000A800750D8A40A820A50D8B4B0EF16F0B0
:102CB000030AD8B469EF16F00AB064EF16F006AE56
:102CC000AEEF16F0ACEF16F002AEACEF16F0AEEFD2
:102CD00016F00250800B0A6E029E0650800B069E74
:102CE0000A18D8B47AEF16F00A50D8B4ACEF16F040
:102CF000AEEF16F00750035CD8B484EF16F0D8A0FE
:102D0000A0EF16F0A6EF16F00650025CD8B48EEFD6
:102D100016F0D8A0A0EF16F0A6EF16F00550015C53
:102D2000D8B498EF16F0D8A0A0EF16F0A6EF16F0E2
:102D30000450005CD8B4B0EF16F0D8B0A6EF16F08F
:102D40000A52D8B4AEEF16F0ACEF16F00A52D8B46F
:102D5000ACEF16F0AEEF16F0D8801200D89012004B
:102D6000D880D884120012000450000A08E10550EF
:102D7000000A05E1FF0E006E7F0E016E58D00D6A4D
:102D8000096A086A01500010D8B4000C01500518F7
:102D90000A6E0ABE0D1E0B6A05AE05D0041E051E86
:102DA000042AD8B4052A01AE05D0001E011E002A4F
:102DB000D8B4012A015005100A6E0ABE10D070EC7A
:102DC0000AF00BB020D00DAE000C001E011E002A30
:102DD000D8B4012A081E091E082AD8B4092A000CF2
:102DE00005AE0DD001BE07D00150096E0050086E2F
:102DF000016A006AE8D7016A006A002A000C011E15
:102E0000001E0B2ADDD7082AD8B4092A0450085C12
:102E1000D8A4D9D70550095CD8A4D5D7096A086ABF
:102E2000002AD8B4012A01AECED70000FF0C120050
:102E300003500718D8A42CEF17F002500618D8A496
:102E40002CEF17F001500518D8A42CEF17F0005004
:102E50000418D8B4D8841200D8941200120052EC8E
:102E600011F000C0FFF0500E0101276F630E286FB4
:102E7000000E296F63DE00C000F10001FF51005C0D
:102E800003E2FFC000F002D000C100F01200000118
:102E9000CD51000A0CE16D6A696A16EC05F0FDEC93
:102EA00011F06DB602D06D86FCD7010ECD6F120009
:102EB00000C008F00150006E016A026A036A0B6AE2
:102EC0000C6A016A026A036A960E036E0A6A00AE11
:102ED00070EF17F0081E001E082AD8B4002A0A8EC8
:102EE00000C001F008C000F0086A026AB1EC11F0FD
:102EF000120001011F6B206B136B146B03C100F0F8
:102F000004C101F005C102F0010E0327000E0423E5
:102F1000052300C0F6FF01C0F7FF02C0F8FF09005B
:102F2000F5CF00F000C010F10052D8B48BEF27F0BD
:102F30001051250A0BE001C1E1FF02C1E2FF10C1FF
:102F4000E6FF014B022B1F4B202BD8D7116B126BC6
:102F5000136B146B23D01387010E0327000E042379
:102F6000052359D01381010E0327000E04230523E6
:102F700052D01383010E0327000E042305234BD0E8
:102F80001487010E0327000E0423052344D0138564
:102F9000010E0327000E042305233DD003C1F6FFD5
:102FA00004C1F7FF05C1F8FF0900F5CF01F001509A
:102FB0002D0AD1E003C1F6FF04C1F7FF05C1F8FFF8
:102FC0000900F5CF01F00150200ACCE003C1F6FF63
:102FD00004C1F7FF05C1F8FF0900F5CF01F001506A
:102FE0002B0AC7E003C1F6FF04C1F7FF05C1F8FFD4
:102FF0000900F5CF01F00150230AC2E003C1F6FF3A
:1030000004C1F7FF05C1F8FF0900F5CF01F0015039
:10301000300ABDE001D09ED713A301D0139113A7AE
:1030200001D0139503C1F6FF04C1F7FF05C1F8FFF6
:103030000900F5CF00F0000E016E00C027F1F1ECA1
:1030400011F0005236E0116B126B11C100F012C189
:1030500001F00A0E046E000E056E0EEC00F003C1C6
:10306000F6FF04C1F7FF05C1F8FF0900F5CF02F034
:1030700002500024116F000E0120126F300E115FFC
:10308000000E125B010E0327000E0423052303C16B
:10309000F6FF04C1F7FF05C1F8FF0900F5CF00F006
:1030A000000E016E00C027F1F1EC11F00052CDE1ED
:1030B00033D003C1F6FF04C1F7FF05C1F8FF0900D3
:1030C000F5CF01F001502A0A27E106C1E9FF07C147
:1030D000EAFFEECF00F0EECF01F000C0E9FF01C043
:1030E000EAFFEECF11F1EECF12F106C1E9FF07C101
:1030F000EAFF020EEE24006E000EEE20016E06C105
:10310000E1FF07C1E2FF00C0E6FF01C0E6FF010EDC
:103110000327000E0423052303C1F6FF04C1F7FFB4
:1031200005C1F8FF0900F5CF01F001502E0A70E14A
:10313000010E0327000E0423052303C1F6FF04C17B
:10314000F7FF05C1F8FF0900F5CF01F001502A0A89
:1031500028E106C1E9FF07C1EAFFEECF00F0EECF9C
:1031600001F000C0E9FF01C0EAFFEECF0EF1EECFA3
:103170000FF106C1E9FF07C1EAFF020EEE24006E5F
:10318000000EEE20016E06C1E1FF07C1E2FF00C0A4
:10319000E6FF01C0E6FF010E0327000E042305230E
:1031A00036D00E6B0F6B03C1F6FF04C1F7FF05C1EC
:1031B000F8FF0900F5CF00F0000E016E00C027F106
:1031C000F1EC11F0005223E00EC100F00FC101F04C
:1031D0000A0E046E000E056E0EEC00F003C1F6FF41
:1031E00004C1F7FF05C1F8FF0900F5CF02F0025056
:1031F00000240E6F000E01200F6F300E0E5F000EC8
:103200000F5B010E0327000E04230523CCD703D048
:103210000E6B0F6B148903C100F004C101F005C1EE
:1032200002F0010E0327000E0423052300C0F6FF61
:1032300001C0F7FF02C0F8FF0900F5CF10F1F9D087
:103240001FC100F020C101F08FEF27F01389E3D7F1
:1032500014852ED1138B14812BD1148329D1138D76
:1032600027D126D1138B138F23D106C1E9FF07C1C4
:10327000EAFFEECF00F0EECF01F000C0E9FF01C0A1
:10328000EAFFEECF1BF1EECF1CF106C1E9FF07C14B
:10329000EAFF020EEE24006E000EEE20016E06C163
:1032A000E1FF07C1E2FF00C0E6FF01C0E6FF000E3C
:1032B0001C1902E1000E1B1904E12E0E1B6F000EFB
:1032C0001C6F1D6B1E6B1D511B25E96E1E511C21B1
:1032D000EA6EEE520BE0010E1D25006E000E1E215F
:1032E000016E00C01DF101C01EF1EDD70E510F118E
:1032F0000AE01E510F5D02E11D510E5D04E20EC198
:103300001DF10FC11EF112511E5D02E111511D5D33
:1033100005E21D51115F1E51125B02D0116B126B41
:1033200013B716D011C100F012C101F0010E115FE8
:10333000000E125B005001100BE001C1E1FF02C161
:10334000E2FF200EE66E014B022B1F4B202BEAD72B
:103350001DC102F01EC103F0010E1D5D006E000EC6
:103360001E59016E00C01DF101C01EF10250031074
:1033700019E01BC1E9FF1CC1EAFF01C1E1FF02C165
:10338000E2FFEECFE6FF014B022B010E1B25006E84
:10339000000E1C21016E00C01BF101C01CF11F4B6F
:1033A000202BD6D713A716D011C100F012C101F0FF
:1033B000010E115F000E125B005001100BE001C105
:1033C000E1FF02C1E2FF200EE66E014B022B1F4B14
:1033D000202BEAD793D506C1E9FF07C1EAFFEECF5C
:1033E00000F0EECF01F000C0E9FF01C0EAFFEECF30
:1033F00010F106C1E9FF07C1EAFF020EEE24006EDC
:10340000000EEE20016E06C1E1FF07C1E2FF00C021
:10341000E6FF01C0E6FF100E1B6F010E1C6F010ED0
:103420001D6F000E1E6F62D7C00E1313000E141313
:103430003FD01051000AD8B403D710516C0AD8B449
:1034400005D710514C0AD8B401D71051660AD8B428
:10345000FFD61051450AD8B4FDD61051650AD8B42C
:10346000FAD61051670AD8B4F8D610516F0AD8B4FA
:10347000F6D61051640AD8B4F4D61051690AD8B4FB
:10348000F0D61051700AD8B4EDD61051580AD8B4FD
:10349000E9D61051780AD8B4E6D61051730AD8B4D8
:1034A000E4D61051630A97E01051750ABDE0B3D716
:1034B000000E1315006E1451070B016E0050011021
:1034C000D8B432EF23F014A904D0060E0E6F000E0C
:1034D0000F6F06C1E9FF07C1EAFFEECF00F0EECFA4
:1034E00001F000C0E9FF01C0EAFFEECF15F1EECF19
:1034F00016F1EECF17F1EECF18F106C1E9FF07C1C3
:10350000EAFF040EEE24006E000EEE20016E06C1EE
:10351000E1FF07C1E2FF00C0E6FF01C0E6FF046A69
:10352000056A066A076A15C100F016C101F017C1E5
:1035300002F018C103F04DEC16F0010ED8B0000EE9
:10354000006E005205E0177F030E1313000E1413D4
:10355000196B1A6B15C100F016C101F017C102F00A
:1035600018C103F0046A056A066A076A61DC000E86
:10357000D8A4010E006E0052D8B48AD018C100F051
:10358000016A026A036AFF0E0016000E01167E0E23
:10359000005E000E015A00C019F101C01AF1010EBF
:1035A000005E000E015A00C019F101C01AF1030EAD
:1035B000046E000E056E0EEC00F000C019F101C0A3
:1035C0001AF10A0E046E000E056EB4EC16F000C07F
:1035D00019F101C01AF1800E0118026E800E025C12
:1035E00002E1000E005C05E2010E0101195F000E10
:1035F0001A5B010119510008276FC0EC12F015C1C8
:1036000004F016C105F017C106F018C107F055EC1B
:1036100009F000C01BF101C01CF102C01DF103C084
:103620001EF1000E046E000E056E000E066E7F0E7B
:10363000076E1BC100F01CC101F01DC102F01EC1CC
:1036400003F04DEC16F0010ED8B0000E006E0052E3
:1036500005E0010E195F000E1A5B1AD0000E046E11
:10366000000E056E200E066E820E076E1BC100F066
:103670001CC101F01DC102F01EC103F04DEC16F09B
:10368000000ED8B0010E006E005202E0194B1A2B4A
:10369000800E006E800E1A19005C02E119510008BC
:1036A00003E3010E106F02D019C110F114B118D04C
:1036B00014A315D0800E1A19006E7F0E005C02E173
:1036C000FC0E195D0BE3800E1A19006E800E0F19A7
:1036D000005C02E10E51195D01E201D001D0F4D38A
:1036E0000E510F1106E014A304D0010E0E5F000E60
:1036F0000F5B000E006E0F51005C02E10E510808D6
:1037000003E2080E106F02D00EC110F115C100F0D7
:1037100016C101F017C102F018C103F0046A056A6E
:10372000066A076A18EC17F0000ED8A4010E006EA6
:103730000052D8B44BD119C127F1C0EC12F000C02F
:1037400004F001C005F002C006F003C007F015C187
:1037500000F016C101F017C102F018C103F002EC2D
:1037600012F000C015F101C016F102C017F103C03C
:1037700018F1010110510008276FC0EC12F000C0D1
:1037800004F001C005F002C006F003C007F015C147
:1037900000F016C101F017C102F018C103F002ECED
:1037A00012F000C021F101C022F102C023F103C0D8
:1037B00024F121C115F122C116F123C117F124C151
:1037C00018F121C100F022C101F023C102F024C18F
:1037D00003F009EC0BF0C9EC0FF000C004F001C0DD
:1037E00005F002C006F003C007F021C100F022C1BD
:1037F00001F023C102F024C103F0EDEC11F0000E42
:10380000046E000E056E000E066E7E0E076E4DEC09
:1038100016F0000ED8B0010E006E00521AE015C16D
:1038200000F016C101F017C102F018C103F0000E3C
:10383000046E000E056E000E066E7E0E076E42ECE4
:1038400007F000C015F101C016F102C017F103C066
:1038500018F115C100F016C101F017C102F018C12E
:1038600003F009EC0BF001011051010F096E0A6A17
:10387000000E0A2209C004F00AC005F0000E0ABEBC
:10388000FF0E066E076E04360490053606360736C0
:1038900004360490053606360736790E0424F66E93
:1038A000630E0520F76E000E0620F86E0900F5CFB6
:1038B00005F00900F5CF06F00900F5CF07F0090083
:1038C000F5CF08F00850035C08E10750025C05E101
:1038D0000650015C02E10550005C1EE3010115C1C8
:1038E00000F016C101F017C102F018C103F0CD0EAF
:1038F000046ECC0E056E4C0E066E7B0E076E55ECFC
:1039000009F000C015F101C016F102C017F103C0A3
:1039100018F1194B1A2B5AD015C100F016C101F03D
:1039200017C102F018C103F009EC0BF010C104F04C
:10393000000E056E066E076E0436049005360636D8
:10394000073604360490053606360736790E042409
:10395000F66E630E0520F76E000E0620F86E090065
:10396000F5CF05F00900F5CF06F00900F5CF07F017
:103970000900F5CF08F00850035C08E10750025C2D
:1039800005E10650015C02E10550005C1FE2010107
:1039900015C100F016C101F017C102F018C103F003
:1039A000000E046E000E056E200E066E820E076E6F
:1039B00055EC09F000C015F101C016F102C017F175
:1039C00003C018F1010E195F000E1A5B010114A368
:1039D00093D014B791D0800E000A006E800E0F199C
:1039E000005C02E10E510A0804E20A0E0E6F000E9E
:1039F0000F6F15C100F016C101F017C102F018C118
:103A000003F009EC0BF000C01BF101C01CF102C077
:103A10001DF103C01EF11B511C111D111E1142E0AE
:103A20000A0E046E000E056E066E076E1BC100F0D6
:103A30001CC101F01DC102F01EC103F0DCEC0FF04F
:103A400008C000F009C001F00AC002F00BC003F08A
:103A5000000E046E031808E10450021805E104503A
:103A6000011802E10050000A1DE1010E0E5F000E78
:103A70000F5B0A0E046E000E056E066E076E1BC10C
:103A800000F01CC101F01DC102F01EC103F0DCEC0E
:103A90000FF000C01BF101C01CF102C01DF103C0FA
:103AA0001EF1B9D7800E0F19006E800E005C02E186
:103AB00010510E5D21E20E51105D276FC0EC12F027
:103AC00000C004F001C005F002C006F003C007F01A
:103AD00015C100F016C101F017C102F018C103F0C2
:103AE00002EC12F000C015F101C016F102C017F18E
:103AF00003C018F10EC110F1050E01010E25006E74
:103B0000000E0F21016E0050115F0150125B0E512B
:103B10000F1103E114B701D004D0010E115F000EA4
:103B2000125B030E1315006E14C101F0000E011696
:103B30000050011004E0010E115F000E125B13A58E
:103B40003CD013A315D013A104D02D0E0001FF6F9C
:103B500003D000012B0EFF6F01C1E1FF02C1E2FFA4
:103B6000FFC0E6FF0101014B022B1F4B202B0CD0A5
:103B700013A10AD001C1E1FF02C1E2FF200EE66EEF
:103B8000014B022B1F4B202B800E006E800E121952
:103B9000005C02E1115100080FE201C1E1FF02C126
:103BA000E2FF300EE66E014B022B1F4B202B010E65
:103BB000115F000E125BE8D73AD013B718D0800E11
:103BC000006E800E1219005C02E1115100080FE234
:103BD00001C1E1FF02C1E2FF200EE66E014B022BA4
:103BE0001F4B202B010E115F000E125BE8D713A3B1
:103BF00012D013A103D02D0E006F02D02B0E006F38
:103C000001C1E1FF02C1E2FF00C1E6FF014B022B4F
:103C10001F4B202B0CD013A10AD001C1E1FF02C120
:103C2000E2FF200EE66E014B022B1F4B202B15C12D
:103C300000F016C101F017C102F018C103F009EC41
:103C40000BF000C01BF101C01CF102C01DF103C04C
:103C50001EF110C100F0000E016E026E036E003600
:103C600000900136023603360036009001360236E7
:103C70000336790E0024F66E630E0120F76E000EF7
:103C80000220F86E0900F5CF04F00900F5CF05F029
:103C90000900F5CF06F00900F5CF07F01BC100F0D1
:103CA0001CC101F01DC102F01EC103F0DCEC0FF0DD
:103CB000300E002601C1E1FF02C1E2FF00C0E6FFB5
:103CC000014B022B1F4B202B0E510F1103E114B798
:103CD00001D06FD001C1E1FF02C1E2FF2E0EE66EFE
:103CE000014B022B1F4B202B10510E5F000E0F5B60
:103CF00010534DE0100710C100F0000E016E026E6F
:103D0000036E00360090013602360336003600900E
:103D1000013602360336790E0024F66E630E01205A
:103D2000F76E000E0220F86E0900F5CF04F00900CE
:103D3000F5CF05F00900F5CF06F00900F5CF07F043
:103D40001BC100F01CC101F01DC102F01EC103F037
:103D5000DCEC0FF00A0E046E000E056E066E076EA8
:103D6000DCEC0FF008C000F009C001F00AC002F05E
:103D70000BC003F0300E002601C1E1FF02C1E2FFDB
:103D800000C0E6FF014B022B1F4B202BB1D70E5179
:103D90000F110FE001C1E1FF02C1E2FF300EE66E3C
:103DA000014B022B1F4B202B010E0E5F000E0F5BF1
:103DB000EED713AB0BD001C1E1FF02C1E2FF450E0C
:103DC000E66E014B022B1F4B202B0AD001C1E1FFF5
:103DD00002C1E2FF650EE66E014B022B1F4B202B4A
:103DE000800E1A19006E800E005C02E1000E195D53
:103DF00011E219510008196F1A51000E1A5701C12A
:103E0000E1FF02C1E2FF2D0EE66E014B022B1F4BBC
:103E1000202B0AD001C1E1FF02C1E2FF2B0EE66EAA
:103E2000014B022B1F4B202B0A0E046E000E056E59
:103E300019C100F01AC101F0B4EC16F0300E0026E2
:103E400001C1E1FF02C1E2FF00C0E6FF0101014B39
:103E5000022B1F4B202B0A0E046E000E056E19C19B
:103E600000F01AC101F0B4EC16F008C000F009C06F
:103E700001F0300E002601C1E1FF02C1E2FF00C0E7
:103E8000E6FF0101014B022B1F4B202B13A71AD079
:103E9000800E006E800E1219005C02E111510008C4
:103EA00011E201C1E1FF02C1E2FF200EE66E014B0B
:103EB000022B1F4B202B010E115F000E125B1151C4
:103EC0001211EFE17EEF17F014A3F3D0800E1A1950
:103ED000006E800E005C02E1000E195D0AE2010E28
:103EE000195D006E000E1A59016E00500E5F0150F0
:103EF0000F5B15C100F016C101F017C102F018C127
:103F000003F009EC0BF000C01BF101C01CF102C072
:103F10001DF103C01EF1010E106F10510A0A34E0AA
:103F200010C100F0000E016E026E036E00360090AC
:103F3000013602360336003600900136023603366B
:103F4000790E0024F66E630E0120F76E000E02203B
:103F5000F86E0900F5CF01F00900F5CF02F0090075
:103F6000F5CF03F00900F5CF04F004501E5D08E121
:103F700003501D5D05E102501C5D02E101501B5D17
:103F800001E202D0102BC9D710510E5D256F000E33
:103F90000F59266F25C10EF126C10FF11BC100F08C
:103FA0001CC101F01DC102F01EC103F0C9EC0FF0ED
:103FB00000C004F001C005F002C006F003C007F025
:103FC00015C100F016C101F017C102F018C103F0CD
:103FD000EDEC11F000C021F101C022F102C023F18B
:103FE00003C024F125C127F1C0EC12F021C104F077
:103FF00022C105F023C106F024C107F055EC09F0F9
:10400000000E046E000E056E000E066E7E0E076E2C
:1040100042EC07F009EC0BF000C01BF101C01CF1F1
:1040200002C01DF103C01EF10E510F1142E00A0E35
:10403000046E000E056E066E076E1BC100F01CC1FB
:1040400001F01DC102F01EC103F0DCEC0FF008C04E
:1040500000F009C001F00AC002F00BC003F0000E2E
:10406000046E031808E10450021805E10450011819
:1040700002E10050000A1DE10A0E046E000E056EFA
:10408000066E076E1BC100F01CC101F01DC102F0DD
:104090001EC103F0DCEC0FF000C01BF101C01CF1ED
:1040A00002C01DF103C01EF1010E0E5F000E0F5B7A
:1040B000BBD7800E006E800E0F19005C02E10E511E
:1040C0000C0816E30EC127F1E8EC0DF015C104F061
:1040D00016C105F017C106F018C107F042EC07F051
:1040E00000C015F101C016F102C017F103C018F1AC
:1040F00015C100F016C101F017C102F018C103F09C
:10410000046A056A066A076A18EC17F0000ED8A45C
:10411000010E006E0052D8B477D015C100F016C160
:1041200001F017C102F018C103F009EC0BF0000E0A
:10413000046E031808E10450021805E10450011848
:1041400002E10050000A60E1800E006E800E1A1934
:10415000005C02E11951010857E219C127F1C0ECD6
:1041600012F000C004F001C005F002C006F003C068
:1041700007F015C100F016C101F017C102F018C117
:1041800003F002EC12F05F0E046E700E056E090E65
:10419000066E810E076E4DEC16F0010ED8B0000EC3
:1041A000006E005206E0090E0101195F000E1A5B55
:1041B00005D00101080E195F000E1A5B19C127F125
:1041C000C0EC12F000C004F001C005F002C006F01F
:1041D00003C007F015C100F016C101F017C102F0CD
:1041E00018C103F002EC12F009EC0BF000C01BF157
:1041F00001C01CF102C01DF103C01EF10101156BCD
:10420000166B176B186B38D015C100F016C101F092
:1042100017C102F018C103F009EC0BF000C01BF14C
:1042200001C01CF102C01DF103C01EF11BC100F052
:104230001CC101F01DC102F01EC103F0C9EC0FF05A
:1042400000C004F001C005F002C006F003C007F092
:1042500015C100F016C101F017C102F018C103F03A
:10426000EDEC11F000C015F101C016F102C017F11C
:1042700003C018F1196B1A6B010E106F10510A0A66
:1042800034E010C100F0000E016E026E036E0036C5
:1042900000900136023603360036009001360236B1
:1042A0000336790E0024F66E630E0120F76E000EC1
:1042B0000220F86E0900F5CF01F00900F5CF02F0F9
:1042C0000900F5CF03F00900F5CF04F004501E5D9E
:1042D00008E103501D5D05E102501C5D02E1015043
:1042E0001B5D01E202D0102BC9D710510E25006EC4
:1042F000000E0F21016E195100261A5101220050A3
:10430000115F0150125B14B704D00E510F1101E17F
:1043100004D0010E115F000E125B030E1315006E28
:1043200014C101F0000E01160050011004E0010E4E
:10433000115F000E125B13A539D013A312D013A185
:1043400003D02D0E086F02D02B0E086F01C1E1FFC4
:1043500002C1E2FF08C1E6FF014B022B1F4B202BDD
:104360000CD013A10AD001C1E1FF02C1E2FF200E6F
:10437000E66E014B022B1F4B202B800E006E800E31
:104380001219005C02E1115100080FE201C1E1FFC6
:1043900002C1E2FF300EE66E014B022B1F4B202BB9
:1043A000010E115F000E125BE8D73AD013B718D098
:1043B000800E006E800E1219005C02E1115100089F
:1043C0000FE201C1E1FF02C1E2FF200EE66E014BE8
:1043D000022B1F4B202B010E115F000E125BE8D742
:1043E00013A312D013A103D02D0E096F02D02B0EF0
:1043F000096F01C1E1FF02C1E2FF09C1E6FF014B04
:10440000022B1F4B202B0CD013A10AD001C1E1FFBE
:1044100002C1E2FF200EE66E014B022B1F4B202B48
:1044200010C100F0100700524CE010C100F0000E67
:10443000016E026E036E00360090013602360336BE
:1044400000360090013602360336790E0024F66EEF
:10445000630E0120F76E000E0220F86E0900F5CF02
:1044600004F00900F5CF05F00900F5CF06F00900CA
:10447000F5CF07F01BC100F01CC101F01DC102F017
:104480001EC103F0DCEC0FF00A0E046E000E056E88
:10449000066E076EDCEC0FF008C000F009C001F0FA
:1044A0000AC002F00BC003F0300E002601C1E1FF8C
:1044B00002C1E2FF00C0E6FF014B022B1F4B202B85
:1044C000AFD7800E006E800E1A19005C02E1195100
:1044D00000080FE201C1E1FF02C1E2FF300EE66E0B
:1044E000014B022B1F4B202B010E195F000E1A5B94
:1044F000E8D7800E000A006E800E0F19005C02E102
:104500000E51080803E2080E106F02D00EC110F120
:1045100010510E5F000E0F5B105303E114B701D072
:104520000AD001C1E1FF02C1E2FF2E0EE66E014B8F
:10453000022B1F4B202B10C127F1C0EC12F015C12C
:1045400004F016C105F017C106F018C107F055ECCC
:1045500009F039EC0DF000C01BF101C01CF102C0E4
:104560001DF103C01EF110534DE0100710C100F003
:10457000000E016E026E036E0036009001360236A8
:10458000033600360090013602360336790E0024D9
:10459000F66E630E0120F76E000E0220F86E090021
:1045A000F5CF04F00900F5CF05F00900F5CF06F0CE
:1045B0000900F5CF07F01BC100F01CC101F01DC1BF
:1045C00002F01EC103F0DCEC0FF00A0E046E000EC8
:1045D000056E066E076EDCEC0FF008C000F009C037
:1045E00001F00AC002F00BC003F0300E002601C13A
:1045F000E1FF02C1E2FF00C0E6FF014B022B1F4BAF
:10460000202BB1D70E510F110FE001C1E1FF02C104
:10461000E2FF300EE66E014B022B1F4B202B010EEA
:104620000E5F000E0F5BEED713A71AD0800E006E40
:10463000800E1219005C02E11151000811E201C163
:10464000E1FF02C1E2FF200EE66E014B022B1F4B81
:10465000202B010E115F000E125B11511211EFE1C0
:104660007EEF17F0C00E1315016E14C102F0000E9C
:104670000216000E021802E1000E0118D8A480D024
:1046800013A927D006C1E9FF07C1EAFFEECF00F06A
:10469000EECF01F000C0E9FF01C0EAFFEECF1BF151
:1046A000EECF1CF1EECF1DF1EECF1EF106C1E9FFFA
:1046B00007C1EAFF040EEE24006E000EEE20016E2C
:1046C00006C1E1FF07C1E2FF00C0E6FF01C0E6FF4F
:1046D0002FD006C1E9FF07C1EAFFEECF00F0EECF11
:1046E00001F000C0E9FF01C0EAFFEECF00F0EECF1D
:1046F00001F0000E01BEFF0E026E036E00C01BF142
:1047000001C01CF102C01DF103C01EF106C1E9FF8A
:1047100007C1EAFF020EEE24006E000EEE20016ECD
:1047200006C1E1FF07C1E2FF00C0E6FF01C0E6FFEE
:10473000800E1E19006E800E005C08E1000E1D5DEB
:1047400005E1000E1C5D02E1000E1B5D18E2030E88
:104750001313000E1413006A016A026A036A1B51E4
:10476000005E1C51015A1D51025A1E51035A00C0CD
:104770001BF101C01CF102C01DF103C01EF14ED09F
:1047800013A927D006C1E9FF07C1EAFFEECF00F069
:10479000EECF01F000C0E9FF01C0EAFFEECF1BF150
:1047A000EECF1CF1EECF1DF1EECF1EF106C1E9FFF9
:1047B00007C1EAFF040EEE24006E000EEE20016E2B
:1047C00006C1E1FF07C1E2FF00C0E6FF01C0E6FF4E
:1047D00025D006C1E9FF07C1EAFFEECF00F0EECF1A
:1047E00001F000C0E9FF01C0EAFFEECF1BF1EECF00
:1047F0001CF1000E1D6F1E6F06C1E9FF07C1EAFF25
:10480000020EEE24006E000EEE20016E06C1E1FFE6
:1048100007C1E2FF00C0E6FF01C0E6FF000E0F196E
:1048200002E1000E0E190FE1000E006E1E1908E1E4
:1048300000501D1905E100501C1902E11B51000A2E
:1048400002E10E4B0F2BC00E1315006E00C005F0D9
:10485000AED0010E106F10510A0A34E010C100F002
:10486000000E016E026E036E0036009001360236B5
:10487000033600360090013602360336790E0024E6
:10488000F66E630E0120F76E000E0220F86E09002E
:10489000F5CF01F00900F5CF02F00900F5CF03F0E4
:1048A0000900F5CF04F004501E5D08E103501D5DC2
:1048B00005E102501C5D02E101501B5D01E202D0E6
:1048C000102BC9D782D0010E106F1051080A34E0A6
:1048D00010C100F0000E016E026E036E00360090F3
:1048E00001360236033600360090013602360336B2
:1048F000080E0024F66E640E0120F76E000E0220F2
:10490000F86E0900F5CF01F00900F5CF02F00900BB
:10491000F5CF03F00900F5CF04F004501E5D08E167
:1049200003501D5D05E102501C5D02E101501B5D5D
:1049300001E202D0102BC9D748D0010E106F1051E0
:104940000C0A34E010C100F0000E016E026E036E1E
:1049500000360090013602360336003600900136EC
:1049600002360336200E0024F66E630E0120F76E29
:10497000000E0220F86E0900F5CF01F00900F5CF16
:1049800002F00900F5CF03F00900F5CF04F0045060
:104990001E5D08E103501D5D05E102501C5D02E152
:1049A00001501B5D01E202D0102BC9D70ED005507B
:1049B000000AD8B44ED70550C00AD8B44AD705501B
:1049C000800A81E00550400AB8E0800E006E800E3B
:1049D0000F19005C02E10E51105D03E20EC110F1EF
:1049E0000DD0800E0F19006E800E005C02E1105198
:1049F0000E5D04E210C10EF1000E0F6F1151121185
:104A00000EE0030E1315006E14C101F0000E011626
:104A10000050011004E0010E115F000E125B800EC9
:104A20000F19006E800E1219005C02E111510E5D2B
:104A300005E20E51115F0F51125B02D0116B126B28
:104A4000C40E1315016E1451080B026E0250080AB1
:104A500002E1400E011808E11151121104E0010EAB
:104A6000115F000E125B1CD0C00E1315016E1451A5
:104A7000080B026E0250080A02E1800E011810E1D4
:104A8000800E006E800E1219005C02E111510208C6
:104A900005E2020E115F000E125B02D0116B126B69
:104AA00013A55DD013A312D013A103D02D0E0A6F4E
:104AB00002D02B0E0A6F01C1E1FF02C1E2FF0AC161
:104AC000E6FF014B022B1F4B202B34D013A10BD040
:104AD00001C1E1FF02C1E2FF200EE66E014B022B95
:104AE0001F4B202B27D0C00E1315016E1451080B3D
:104AF000026E0250080A02E1800E01181BE101C19A
:104B0000E1FF02C1E2FF300EE66E014B022B1F4BAC
:104B1000202B13AB03D0580E0B6F02D0780E0B6F07
:104B200001C1E1FF02C1E2FF0BC1E6FF014B022B15
:104B30001F4B202B1151121111E001C1E1FF02C1E5
:104B4000E2FF300EE66E014B022B1F4B202B010EB5
:104B5000115F000E125B11511211EFE174D011516F
:104B6000121113E013B711D001C1E1FF02C1E2FF3E
:104B7000200EE66E014B022B1F4B202B010E115F06
:104B8000000E125B11511211EFE113A312D013A109
:104B900003D02D0E0C6F02D02B0E0C6F01C1E1FF64
:104BA00002C1E2FF0CC1E6FF014B022B1F4B202B81
:104BB0000CD013A10AD001C1E1FF02C1E2FF200E17
:104BC000E66E014B022B1F4B202BC00E1315016EFE
:104BD0001451080B026E0250080A02E1400E01183F
:104BE0000BE101C1E1FF02C1E2FF300EE66E014BB5
:104BF000022B1F4B202B27D0C00E1315016E145112
:104C0000080B026E0250080A02E1800E01181BE137
:104C100001C1E1FF02C1E2FF300EE66E014B022B43
:104C20001F4B202B13AB03D0580E0D6F02D0780E04
:104C30000D6F01C1E1FF02C1E2FF0DC1E6FF014BB3
:104C4000022B1F4B202B800E006E800E0F19005C74
:104C500002E10E51105D0BE201C1E1FF02C1E2FF72
:104C6000300EE66E014B022B1F4B202BECD70EC1F2
:104C700000F00FC101F0010E0E5F000E0F5B00503F
:104C80000110D8B42AD1C00E1315006E00C021F156
:104C90000AD10EC100F00FC101F0000E0FBFFF0ED0
:104CA000026E036E0036009001360236033600367F
:104CB0000090013602360336790E0024F66E630E3C
:104CC0000120F76E000E0220F86E0900F5CF04F007
:104CD0000900F5CF05F00900F5CF06F00900F5CF82
:104CE00007F01BC100F01CC101F01DC102F01EC184
:104CF00003F0DCEC0FF00A0E046E000E056E066E7B
:104D0000076EDCEC0FF008C000F009C001F00AC02B
:104D100002F00BC003F0300E0024106FD3D013ABA1
:104D200045D00EC100F00FC101F0000E0FBFFF0E05
:104D3000026E036E003600900136023603360036EE
:104D40000090013602360336080E0024F66E640E1B
:104D50000120F76E000E0220F86E0900F5CF04F076
:104D60000900F5CF05F00900F5CF06F00900F5CFF1
:104D700007F01BC100F01CC101F01DC102F01EC1F3
:104D800003F0DCEC0FF00F0E0016000E01160216F9
:104D90000316BE0E0024F66E640E0120F76E000EA0
:104DA0000220F86E0900F5CF10F144D00EC100F0DA
:104DB0000FC101F0000E0FBFFF0E026E036E003632
:104DC0000090013602360336003600900136023676
:104DD0000336080E0024F66E640E0120F76E000EF6
:104DE0000220F86E0900F5CF04F00900F5CF05F0B8
:104DF0000900F5CF06F00900F5CF07F01BC100F060
:104E00001CC101F01DC102F01EC103F0DCEC0FF06B
:104E10000F0E0016000E011602160316AD0E00242A
:104E2000F66E640E0120F76E000E0220F86E090087
:104E3000F5CF10F147D00EC100F00FC101F0000E08
:104E40000FBFFF0E026E036E003600900136023671
:104E5000033600360090013602360336200E002459
:104E6000F66E630E0120F76E000E0220F86E090048
:104E7000F5CF04F00900F5CF05F00900F5CF06F0F5
:104E80000900F5CF07F01BC100F01CC101F01DC1E6
:104E900002F01EC103F0DCEC0FF0070E0014106FDF
:104EA000300E10270FD02151000AD8B4F2D621516C
:104EB000C00AD8B4EED62151800AD8B430D72151D7
:104EC000400AB9E001C1E1FF02C1E2FF10C1E6FF03
:104ED000014B022B1F4B202BCAD613A71AD0800ED2
:104EE000006E800E1219005C02E11151000811E2FF
:104EF00001C1E1FF02C1E2FF200EE66E014B022B71
:104F00001F4B202B010E115F000E125B115112116D
:104F1000EFE17EEF17F01FC100F020C101F0120099
:104F20000001FF6B200ECD5D03E36DB201D002D016
:104F3000006A32D0CEC027F1CFC028F1D2EC0DF0FC
:104F4000005229E1CEC005F1CFC006F1000E0001EC
:104F5000CF1902E1000ECE190BE0010E010105256B
:104F6000E96E000E0621EA6EEECF00F000C0FFF001
:104F7000010104C127F1286B01C129F102C12AF105
:104F800003C12BF1A5EC0BF000C0CEF001C0CFF0B7
:104F9000FFC000F001D0006A12000B6A0350D8B4C1
:104FA00013EF28F002500A6E028E8E0E035E03AEDF
:104FB00017EF28F0036C080E035CD8A0F2EF27F07F
:104FC000036E013602C001F0026A080E035CD8A02D
:104FD000F2EF27F0036E0136016A0350D8A4D8908F
:104FE000FCEF27F00350D8B4FCEF27F0D890023242
:104FF0000132032EF6EF27F00BBC01A009EF28F0D9
:10500000D8A009EF28F0012AD8B4022A02BE26EF60
:1050100028F00AAE2CEF28F0021E011E012AD8B497
:10502000022A2CEF28F0026A016A2CEF28F00B808C
:105030000BAE30EF28F0026A0AAE30EF28F0FF0E18
:10504000026E016E0A36023230EF28F0010E0C6E4D
:10505000D8EC06F032EF28F0000E0C6E32EF28F09C
:10506000FF0E0C6E0150006E0250016E1200F00E29
:1050700001010115006E008600C0FFF03EC02DF159
:10508000040E00102E6FB8EC06F000C03FF0000ECA
:10509000406E270E0D6E0D2EFED7000000003EC0A4
:1050A0002DF1FB0E0001FF1501012E6FB8EC06F08B
:1050B00000C03FF0000E406E270E0D6E0D2EFED785
:1050C000000000000101025335E001C100F000368C
:1050D0000090003600900036009000360090F00EF0
:1050E0000016008600C0FFF03EC02DF1040E001037
:1050F0002E6FB8EC06F000C03FF0000E406E070EB9
:105100000D6E0D2EFED7000000003EC02DF1FB0EEF
:105110000001FF1501012E6FB8EC06F000C03FF052
:10512000000E406E4E0E0C6EEB0E0D6E0D2EFED769
:105130000C2EFCD7120001C1F6FF02C1F7FF03C11C
:10514000F8FF0900F5CF00F0005212E001C1F6FFB0
:1051500002C1F7FF03C1F8FF0900F5CF27F169ECA1
:105160000FF0010E01010127000E02230323E3D7F4
:1051700012000101046B056B01C1F6FF02C1F7FFCC
:1051800003C1F8FF0900F5CF01F00150000A1DE04E
:10519000800E0519006E800E005C02E1140E045DA5
:1051A00014E201C1F6FF02C1F7FF03C1F8FF0900D5
:1051B000F5CF27F169EC0FF0010E01010127000E78
:1051C00002230323044B052BD7D71200570E0D6E75
:1051D0000D2EFED7000000001200200E0001CD5D54
:1051E00003E36DB201D002D0006A4DD0E1C027F1D7
:1051F000E2C028F1D2EC0DF0005244E104C127F1E5
:10520000010E286F01C129F102C12AF103C12BF15E
:10521000A5EC0BF000C0E1F001C0E2F00001DB6B97
:10522000DC6BDD6BDE6BE1C027F1E2C028F1D2EC74
:105230000DF0005210E0010E016E0150000A02E173
:1052400035EC0CF00001DB51DC11DD11DE1102E068
:10525000006A19D0E8D70001E1C005F1E2C006F10B
:10526000000EE21902E1000EE1190AE0010E01014F
:105270000525E96E000E0621EA6EEECF00F003D0A0
:10528000006A01D0006A1200ED0E0001F56F000EF9
:10529000F66FE8C001F1E9C002F1EAC003F1EBC02A
:1052A00004F1ECC005F1F50E0101066F000E076F69
:1052B00079EC17F000C0F3F001C0F4F000500001E9
:1052C000E825E16E0150E921E26EE66AF3C000F0E4
:1052D000F4C001F012000050086E0150006E016A27
:1052E000026A036A0B6A0C6A960E036E0A6A00C0B1
:1052F00001F008C000F0086A026AB1EC11F0120077
:10530000D40E0101016F010E026FB1DEE8C001F1A0
:10531000E9C002F1EAC003F12CDF120054D0800E84
:105320000101016F010E026FA2DE710E0101016F1A
:10533000640E026F000E036FFEDE800E0101016F2E
:10534000010E026F94DE58D0C00E0101016F010EF4
:10535000026F8DDE710E0101016F640E026F000E8F
:10536000036FE9DEC00E0101016F010E026F7FDEE7
:1053700043D0940E0101016F010E026F78DE710EB1
:105380000101016F640E026F000E036FD4DE940EF4
:105390000101016F010E026F6ADE2ED0D40E0101F1
:1053A000016F010E026F63DE710E0101016F640E69
:1053B000026F000E036FBFDED40E0101016F010EFC
:1053C000026F55DE19D0000E0001E91902E1010E4D
:1053D000E819A5E0000EE91902E1020EE819B4E0AF
:1053E000000EE91902E1030EE819C3E0000EE91905
:1053F00002E1040EE819D2E01200D2C001F1D3C0DC
:1054000002F1400E0101036F010E046F89DD1200ED
:10541000C26A070EC012C08EE8C000F000360090CD
:10542000003600900050C212C280D0DEC282C2A2FA
:1054300001D0FDD7C4CF01F0006AC3500012000EA6
:105440000112C29012000001CD51010A07E16DBAAC
:1054500005D0686A69806988020ECD6F68A406D09D
:1054600069A404D0FB0E68163AEC07F06DA203D0D5
:10547000C7EC06F0E1D068A019D069A017D0E8EC1D
:1054800009F0040ECD6F200E0401026F040E036FAD
:10549000080E016F000E0015006E00C000F48C0EA7
:1054A0000011006E00C000F4FE0E681668A806D059
:1054B00069A804D045EC0AF0EF0E681668AC04D079
:1054C00069AC02D0BF0E681668AA04D069AA02D0DF
:1054D00027EC0AF068A202D069B26A6A040E0001E1
:1054E000CD5D03E2C7EC06F0A7D069A6A3D0010109
:1054F000336B040E335DD8B09DD068A697D06CCFC7
:10550000D8F0F70E6816780E0001D815016E01501C
:10551000000AD8A48AD0FD0ED815016E026AFF0ECB
:105520000216000E021802E1000E01186EE17E0E56
:10553000D815016E01C003F00332039E03C000F0D2
:10554000000E016E003600900136003600900136E4
:10555000000E0024026E040E0120036E02C0D9F07A
:1055600003C0DAF002C0C8F003C0C9F0040EC819C5
:10557000006E00C0C8F002C0E9FF03C0EAFFEECF32
:1055800000F000C001F03C0E01160132019E013214
:10559000019E01500D0A36E1020ED925E96E000E7A
:1055A000DA21EA6EEECF01F0EECF02F00250040AEB
:1055B00002E1280E011823E1020ED925E16E000E4A
:1055C000DA21E26E200EE66E040EE66E0101326B09
:1055D000080E325D14E2200EE16E040EE26E3251CE
:1055E000E126D8B0E22A280EE96E040EEA6E3251A6
:1055F000E926D8B0EA2AEECFE6FF322BE9D7A0ECB5
:105600000AF002D04AEC0AF00FD00001FD0ED815C6
:10561000016E026AFF0E0216000E021802E1040E6D
:10562000011802E1E6EC06F000D001D003D0010140
:10563000332B5FD7C7EC06F01200CD6ACD8ACD8838
:105640000B0ECF6EDB0ECE6E3B6A3C6A396A3A6A4D
:105650009E909D909F90F29CCD9012000001EE5183
:10566000000805E3070EEF6F000EF06F12D0EE5149
:10567000160805E2170EF16F000EF26F06D0EE511C
:10568000010FF16FF26B000EF223F1C0EFF0F2C0E8
:10569000F0F0EFC0F9F0F0C0FAF0F36BF46B046ACD
:1056A000056A066A076AE8C000F0E9C001F0EAC0CE
:1056B00002F0EBC003F04DEC16F0010ED8B0000E76
:1056C000006E005209E0ECC0E1FFEDC0E2FF2D0EDC
:1056D000E66EEC4BED2BEA7FE8C004F0E9C005F084
:1056E000EAC006F0EBC007F0006A016A026A036ACA
:1056F0004DEC16F0010ED8B0000E006E005237E0EF
:10570000000E046E000E056E000E066E7F0E076E14
:10571000E8C000F0E9C001F0EAC002F0EBC003F01D
:105720004DEC16F0010ED8B0000E006E00521FE0D6
:10573000E8C000F0E9C001F0EAC002F0EBC003F0FD
:10574000000E046E000E056E200E066E820E076EB1
:1057500055EC09F000C0E8F001C0E9F002C0EAF041
:1057600003C0EBF0010EF35F000EF45BC9D7000E2F
:10577000046E000E056E200E066E820E076EE8C0E7
:1057800000F0E9C001F0EAC002F0EBC003F04DEC1C
:1057900016F0000ED8B0010E006E00521EE0000E92
:1057A000046E000E056E200E066E820E076EE8C0B7
:1057B00000F0E9C001F0EAC002F0EBC003F002EC37
:1057C00012F000C0E8F001C0E9F002C0EAF003C046
:1057D000EBF00001F34BF42BCAD7F351F927F45146
:1057E000FA23010EF56F000EF66F010E006E000E2B
:1057F000016E58EC17F000C0FBF001C0FCF002C0D5
:10580000FDF003C0FEF0800EF619006E800EFA194E
:10581000005C02E1F951F55D1EE2000E046E000E1F
:10582000056E200E066E820E076EFBC000F0FCC0F7
:1058300001F0FDC002F0FEC003F002EC12F000C067
:10584000FBF001C0FCF002C0FDF003C0FEF000015F
:10585000F54BF62BD8D7000E046E000E056E000E29
:10586000066E800E076EFBC000F0FCC001F0FDC0AC
:1058700002F0FEC003F002EC12F0E8C004F0E9C050
:1058800005F0EAC006F0EBC007F042EC07F000C0FC
:10589000E8F001C0E9F002C0EAF003C0EBF0000E4E
:1058A000046E000E056E200E066E820E076E4DEC25
:1058B00016F0000ED8B0010E006E00520BE0000E84
:1058C0000001E86F000EE96F000EEA6F7F0EEB6FCC
:1058D000F34BF42B0001800EF419006E800E005C77
:1058E00002E1000EF35D38E2ECC0E1FFEDC0E2FF43
:1058F000300EE66EEC4BED2BECC0E1FFEDC0E2FFAD
:105900002E0EE66EEC4BED2B800EFA19006E800E1B
:10591000005C02E1000EF95D04E2F951F35FFA5117
:10592000F45BFF0EF56FFF0EF66F800EF419006E3C
:10593000800EF619005C02E1F551F35D0DE2ECC05A
:10594000E1FFEDC0E2FF300EE66EEC4BED2B010EF9
:10595000F55F000EF65BE9D7F56BF66B800EF61976
:10596000006E800EFA19005C02E1F951F55D63E208
:10597000E8C000F0E9C001F0EAC002F0EBC003F0BB
:10598000CDEC27F000C0F7F001C0F8F0300E002693
:10599000ECC0E1FFEDC0E2FF00C0E6FFEC4BED2BF9
:1059A000F651F41902E1F351F51908E1ECC0E1FFF9
:1059B000EDC0E2FF2E0EE66EEC4BED2BF7C000F0D3
:1059C000F8C001F058EC17F000C0FBF001C0FCF08B
:1059D00002C0FDF003C0FEF000C004F001C005F0FD
:1059E00002C006F003C007F0E8C000F0E9C001F013
:1059F000EAC002F0EBC003F0EDEC11F000C0E8F0FB
:105A000001C0E9F002C0EAF003C0EBF0000E046E42
:105A1000000E056E200E066E820E076E55EC09F024
:105A200000C0E8F001C0E9F002C0EAF003C0EBF00A
:105A3000F54BF62B93D7ECC0E1FFEDC0E2FFE66A31
:105A400012000001EA6BEB6BE8C0E9FFE9C0EAFF76
:105A5000EE50000A17E0800EEB19006E800E005C1D
:105A600002E1140EEA5D0EE2E8C0E9FFE9C0EAFFD8
:105A7000EECF27F169EC0FF00001E84BE92BEA4B80
:105A8000EB2BE2D712000900F5CFE6FF0006FBE1A1
:105A90000106F9E11200ECC000F00001EC07005231
:105AA00028E0E8C0E9FFE9C0EAFFEE50000A0CE098
:105AB000E8C0E9FFE9C0EAFFEAC0D9FFEBC0DAFFBE
:105AC000EE50DE1801E10FD0E8C0E9FFE9C0EAFFBF
:105AD000EAC0D9FFEBC0DAFFDE50EE5C006E016A6F
:105AE000000E015A08D00001E84BE92BEA4BEB2BE2
:105AF000D2D7006A016A1200E8C002F0E9C003F0E0
:105B000002C000F003C001F0024A032A00C0E9FF0E
:105B100001C0EAFFEE5201E0F3D70001E851025C58
:105B2000006EE9510358016E010E005E000E015A2D
:105B30001200939093928A908A9293809382C79E48
:105B4000C79C380EC66E12004E0E3E6E5C0E0B6E7B
:105B5000510E0C6E600E0D6E0D2EFED70C2EFCD766
:105B60000B2EFAD70000300E0101016F026B37ECEB
:105B700028F0040E0B6E0C0E0C6E330E0D6E0D2EF7
:105B8000FED70C2EFCD70B2EFAD700000000300EEB
:105B90000101016F026B37EC28F0020E0B6E380E1C
:105BA0000C6EAD0E0D6E0D2EFED70C2EFCD70B2EEF
:105BB000FAD7300E0101016F026B37EC28F0020EAC
:105BC0000B6E380E0C6EAD0E0D6E0D2EFED70C2E1C
:105BD000FCD70B2EFAD7200E0101016F026B37ECB8
:105BE00028F0020E0B6E380E0C6EAD0E0D6E0D2EE3
:105BF000FED70C2EFCD70B2EFAD7280E0101016F11
:105C0000010E026F37EC28F0020E0B6E380E0C6E90
:105C1000AD0E0D6E0D2EFED70C2EFCD70B2EFAD727
:105C2000080E0101016F010E026F37EC28F0020E21
:105C30000B6E380E0C6EAD0E0D6E0D2EFED70C2EAB
:105C4000FCD70B2EFAD7010E0101016F010E026F76
:105C500037EC28F0070E0B6E170E0C6E6A0E0D6EE9
:105C60000D2EFED70C2EFCD70B2EFAD70000060EF9
:105C70000101016F010E026F37EC28F0020E0B6E6E
:105C8000380E0C6EAD0E0D6E0D2EFED70C2EFCD701
:105C90000B2EFAD70C0E0101016F010E026F37ECCB
:105CA00028F0020E0B6E380E0C6EAD0E0D6E0D2E22
:105CB000FED70C2EFCD70B2EFAD71200E8C001F14C
:105CC000E9C002F1EAC003F1010E0101046FEDEC3D
:105CD00028F01200FF0E0001826FFF0E836FFF0E8F
:105CE000846FFF0E856FC26A070EC012C08EC2801D
:105CF00012002FEC17F000C0E3F0010ED56FE8C0E2
:105D0000D2F0E9C0D3F0EAC0D6F0EBC0D7F0E8ECAF
:105D100009F0010E016E0150010A02E147EC17F093
:105D2000120000C023F001C022F002C021F003C025
:105D300020F004C01FF005C01EF008C01DF009C00F
:105D40001CF00AC01BF00BC01AF0E1CF2CF0E2CF20
:105D50002DF0E9CF2AF0EACF2BF0F3CF28F0F4CFE3
:105D600029F0F5CF27F0F8CF24F0F7CF25F0F6CFC4
:105D700026F023EC2AF027C0F5FF24C0F8FF25C049
:105D8000F7FF26C0F6FF28C0F3FF29C0F4FF23C0A9
:105D900000F022C001F021C002F020C003F01FC0BB
:105DA00004F01EC005F01DC008F01CC009F01BC0A7
:105DB0000AF01AC00BF02AC0E9FF2BC0EAFF2CC082
:105DC000E1FF2DC0E2FF11007FEC32F0806A92808B
:105DD0009292938093829396070EB46E0A0E0B6E86
:105DE000220E0C6EA10E0D6E0D2EFED70C2EFCD7C2
:105DF0000B2EFAD7780EC86E9CDE8A9689926ADFDF
:105E0000070E0B6E170E0C6E6A0E0D6E0D2EFED762
:105E10000C2EFCD70B2EFAD70000860EC66F000E94
:105E2000C76F080E5B6E000EE86F050EE96F400E3F
:105E3000EA6F050EEB6F5DDFF19E780EC86E79DEBE
:105E4000070E0B6E170E0C6E6A0E0D6E0D2EFED722
:105E50000C2EFCD70B2EFAD7000076DE070E0B6E49
:105E6000170E0C6E6A0E0D6E0D2EFED70C2EFCD783
:105E70000B2EFAD70000010E0001E86F000EE96F4B
:105E80008EEC29F0860E0101016F640E026F000E88
:105E9000036F9BEC28F0020E0001E86F000EE96F23
:105EA0008EEC29F0710E0101016F640E026F000E7D
:105EB000036F9BEC28F03D0E0B6EE10E0C6E3F0E57
:105EC0000D6E0D2EFED70C2EFCD70B2EFAD7000030
:105ED0000000030E0001E86F000EE96F8EEC29F060
:105EE0005C0E0101016F640E026F000E036F9BECEC
:105EF00028F03D0E0B6EE10E0C6E3F0E0D6E0D2E5A
:105F0000FED70C2EFCD70B2EFAD700000000460E51
:105F10000001E86F640EE96F000EEA6F80EC29F073
:105F20003D0E0B6EE10E0C6E3F0E0D6E0D2EFED76C
:105F30000C2EFCD70B2EFAD700000000396A3A6A03
:105F40001DEC2BF09D80CD80F28CF28E400E000176
:105F5000E86F050EE96F280EEA6F640EEB6F000E16
:105F6000EC6F44EC29F0000E3A1802E1000E3918EB
:105F70000BE10001400EE86F050EE96F400EEA6F7D
:105F80009DDE005201E1EFD7FDEC29F0005207E160
:105F9000000E3A1802E1000E391801E1F5D7000EA3
:105FA0003A1802E1010E39185DE1396A3A6A3B6A32
:105FB0003C6A9D800001E86B08EC2AF000C05CF0B0
:105FC00001C05DF06BEC29F0000E046E000E056E52
:105FD000200E066E810E076E55EC09F0000E046E61
:105FE000000E056E000E066E890E076E02EC12F0B2
:105FF00000C061F001C062F002C063F003C064F051
:1060000000C0E8F001C0E9F002C0EAF003C0EBF024
:10601000650E0001EC6F000EED6F020EEE6F2EECC0
:106020002BF0040EE86F000EE96F8EEC29F0C6C06D
:10603000E8F0C7C0E9F0CF0E0001EA6F640EEB6F25
:10604000000EEC6F5CC0EDF05DC0EEF0650EEF6F22
:10605000000EF06F44EC29F0C6C0E8F0C7C0E9F0CC
:10606000F0DCBDD00001030EE86F000EE96F8EEC8E
:1060700029F0000E0001E86F050EE96FE2DC000E6A
:10608000E86F050EE96F38DD00C057F001C058F029
:10609000000E015C02E1140E005C1EE25750940FEA
:1060A0000101016F020E015F010E026F37EC28F053
:1060B00057C059F058C05AF0000E006E5A50005C9C
:1060C00002E15950140808E3200E0101276F69EC22
:1060D0000FF0594A5A2AF0D7000E0001E86F050E5A
:1060E000E96F350EEA6F000EEB6F030EEC6FD3DC39
:1060F000000E011802E1000E001864E10001E86BD7
:1061000008EC2AF000C05CF001C05DF06BEC29F0F7
:10611000000E046E000E056E200E066E810E076ED8
:1061200055EC09F0000E046E000E056E000E066EB2
:10613000890E076E02EC12F000C061F001C062F03F
:1061400002C063F003C064F000C0E8F001C0E9F0F1
:1061500002C0EAF003C0EBF0650E0001EC6F000E28
:10616000ED6F020EEE6F2EEC2BF0400EE86F050E79
:10617000E96FA10EEA6F630EEB6F000EEC6F5CC06F
:10618000EDF05DC0EEF05CC0EFF05DC0F0F0650ECC
:10619000F16F000EF26F44EC29F0400EE86F050E2F
:1061A000E96FAADC00C057F001C058F00001400EB2
:1061B000E86F050EE96F400EEA6F80DD005201E1E5
:1061C000F5D70DD0400E0001E86F050EE96FDF0E28
:1061D000EA6F640EEB6F000EEC6F44EC29F05D503B
:1061E000030802E15C50B60802E28A8601D08A9672
:1061F000000E5D5C02E1320E5C5C02E2898201D03D
:1062000089921F0E0B6E710E0C6E1E0E0D6E0D2EF2
:10621000FED70C2EFCD70B2EFAD70000B5D6FFD731
:1062200000C019F001C018F0156ED8CF16F0E0CFFD
:1062300017F09DA01ED09EA01CD0010E3B24006E26
:10624000000E3C20016E00C03BF001C03CF0000E8F
:106250003C5C02E1180E3B5C07E33B6A3C6A010EC2
:10626000396E000E3A6E9D900B0ECF6EDB0ECE6E29
:106270009E901750E06E1650D86E153A153819C01A
:1062800000F018C001F010000000007F0000208224
:106290000000488500007A8800401C8C0050438F25
:1062A000002474928096189620BC3E99286B6E9CB0
:1062B000F90215A0EC782DC1CAF249E20000007F76
:1062C000CDCC4C7B0AD723786F12037517B7517169
:1062D000ACC5276EBD37066B95BF566777CC2B6470
:1062E0005F700961FFE65B5D08E53C3C6042221B94
:1062F000200355005300420020004800490044009C
:1063000020004C0069006200720061007200790098
:10631000000000000000000000000000000000007D
:106320000100000008000000400000000002000022
:1063300000100000008000000000040000002000A9
:106340000000000100000008000000400000000004
:1063500009022900010100C0320904000002030003
:1063600000000921010100012221000705810340ED
:10637000000107050103400001010000000A0000C0
:106380000064000000E803000010270000A0860160
:106390000040420F008096980000E1F50500CA9A7F
:1063A0003B204144433D25203575202020202530C9
:1063B00034582020736F697420257320566F6C74D5
:1063C00073200D0A0022034D0069006B0072006FFC
:1063D0000065006C0065006B00740072006F006E59
:1063E0000069006B0061000600FF0901A1011901AD
:1063F0002940150026FF00750895408102190129E2
:1064000040750895409102C0010000001000000096
:10641000000100000010000000000100000010005A
:1064200000000001000000102054696D65723120E9
:10643000696E697469616C6973E9206574204172E1
:106440006DE9200D0A0056657273696F6E20313454
:106450002F30352F3230313520202000484944205C
:106460005465726D696E616C205553422050432013
:10647000004D696B726F432050726F2056362E3577
:106480003020202020003138463235353020555319
:10649000422034384D487A202020001201000200AA
:1064A00000000834123412010001020001303132C0
:1064B00033343536373839616263646566003031AC
:1064C000323334353637383941424344454600414A
:1064D00044433D2520357520253673205620004E37
:1064E0006F20636F6D7072656E646F200D0A0028F7
:1064F0006E756C6C2900414443000403090410EEDE
:106500002EF00B0E006E010E016EEF0EF66E640E95
:10651000F76E000EF86E43EC2DF01200FFFFFFFF48
:10652000FFFFFFFFFFFFFFFFFFFFFFFFFFFFFFFF7B
:10653000FFFFFFFFFFFFFFFFFFFFFFFFE4EF2EF076
:10654000CEEC3FF09AEC3EF0000E00019E6F050E7F
:106550009F6F400EA06F050EA16FA2EC3EF0BDEC48
:106560003EF0005206E198EC3EF0BBEC3DF0E6DF79
:1065700002D0EAEC3EF0FFD7800E0001C011006EA1
:1065800000C066F01200C0C063F0C1C064F0C2C0B9
:1065900067F0C3C068F0800E0001C411006E008077
:1065A00000C066F01200000E056E040E066EC0C03C
:1065B00003F0000E046E03360436039003360436EF
:1065C0000390C1C000F0000E016E0036013600904D
:1065D000005003260150042203C001F004C002F061
:1065E00001360190023601360190023601C003F0F7
:1065F00002C004F004320332049E04BC048E043250
:106600000332049E04BC048E03C000F004C001F0F9
:106610000036009001360036009001360550002605
:106620000650012200C005F001C006F000C0E1FFE5
:1066300001C0E2FFE69E0001C151000A12E1C0C0A4
:1066400000F0000E016E003600900136940E00241A
:10665000E16E000E0120E26E05C0E6FF06C0E6FF17
:1066600011D0C0C000F0000E016E0036009001365F
:106670007D0E0024E16E000E0120E26E05C0E6FFF3
:1066800006C0E6FF05C0E1FF06C0E2FFE69C040E7F
:106690000524E16E000E0620E26EE68C1200C0C0FA
:1066A00063F0C1C064F0C2C065F0C3C067F0C4C08D
:1066B00068F0800E0001C511006E00C066F0120087
:1066C0000001BC51000A12E0BBC000F0000E016ED8
:1066D0000036009001367D0E0024E96E000E012088
:1066E000EA6EEECF04F0EECF05F011D0BBC000F0A3
:1066F000000E016E003600900136940E0024E96E03
:10670000000E0120EA6EEECF04F0EECF05F0020E8F
:106710000424E16E000E0520E26EBDC0E6FFBEC09F
:10672000E6FF010E0424E16E000E0520E26EBFC0FC
:10673000E6FF04C0E9FF05C0EAFFEECF00F004C0A9
:10674000E1FF05C0E2FF400E0014E66E04C0E9FF61
:1067500005C0EAFFEECF00F004C0E1FF05C0E2FF94
:10676000880E0010E66EBC51000A1BE0BBC000F0B2
:10677000000E016E0036009001367D0E0024026E80
:10678000000E0120036E02C0E9FF03C0EAFF040E01
:10679000EE18006E02C0E1FF03C0E2FF00C0E6FF9A
:1067A0001AD0BBC000F0000E016E0036009001361A
:1067B000940E0024026E000E0120036E02C0E9FF59
:1067C00003C0EAFF040EEE18006E02C0E1FF03C032
:1067D000E2FF00C0E6FF04C000F005C001F01200B7
:1067E00020C401F01F0E01160150010A01E08BD0F8
:1067F00004012451000A01E086D02151060A38E143
:106800002DD000018B51010A12E1ED0EC06F7E0EFA
:10681000C16F000EC26F120EC027000EC123C2232B
:10682000090EC36F000EC46F400EC56F38DF20D055
:1068300000018B51010A0DE15E0EC06F7F0EC16F2A
:10684000000EC26F210EC36F000EC46F400EC56FE5
:1068500026DF0ED00001C06B8FDE0AD00401235169
:10686000210ACFE02351220AE3E02351230AF2E078
:1068700020C401F0600E0116050E006E005004E009
:106880000132019EFF0FFBD70150010A01E03BD00E
:1068900027D039D038D09D0E0001C06F000EC16FD7
:1068A000010EC26F000EC36F400EC46F6CDE2BD0A2
:1068B0000001C06B61DE23C49DF025D000019C0E59
:1068C000C06F000EC16F010EC26F000EC36FC46BAC
:1068D0005ADE19D00001C06B4FDE22C49CF013D0E9
:1068E00004012151010AD5E02151090AD3E02151C7
:1068F000020AD1E021510A0ADBE02151030ADEE05D
:1069000021510B0AE7E01200700EE16E0F0EE26EED
:106910000001BB51E126D8B0E22ABCC0E6FFBCA50D
:1069200004D0BBC0C0F0C16B3EDEBCA305D0BBC071
:10693000C0F0010EC16F37DE12000001865314E073
:10694000010EBB6F1E0EBC6FDFDF010EBB6FBC6B99
:106950009AC0BDF09BC0BEF0400EBF6FB1DE00C05C
:1069600098F001C099F013D0010EBB6F1E0EBC6FE2
:10697000CBDF010EBB6FBC6B9AC0BDF09BC0BEF0FD
:10698000400EBF6F9DDE00C098F001C099F012006C
:106990000001865301E024DF1200B5C002F0B6C04A
:1069A00003F0B8C000F0B9C001F0010E0001B85FFB
:1069B000000EB95B0050011009E002C0E1FF03C006
:1069C000E2FFB7C0E6FF024A032AEBD712000CD061
:1069D000B4DF3CD03BD0DCDF39D038D037D036D034
:1069E00035D0000033D032D0000E0001B61902E1DC
:1069F000010EB519EDE0000EB61902E1020EB5194F
:106A0000E9E0000EB61902E1030EB519E4E0B65153
:106A1000000A02E1730EB519E0E0B651000A02E186
:106A2000750EB519DBE0B651000A02E1740EB51916
:106A3000D6E0B6513F0A02E1FF0EB519D1E0B651DA
:106A4000000A02E1720EB519CCE0CDD7010E006E3E
:106A500012000B6A0A6A096A00500402F4CF09F0B6
:106A6000F3CF08F001500502F4CF0BF0F3CF0AF09A
:106A700000500502F3500926F4500A22E86A0B225E
:106A800001500402F3500926F4500A22E86A0B224E
:106A900008C000F009C001F00AC002F00BC003F00A
:106AA00012000401286B296B4AD00001668F040193
:106AB000288100018451010A02E10401288354D095
:106AC0000001668F51D00001668F040124BF16D0EB
:106AD00024C403F00F0E031603C000F0000E016E75
:106AE000003600900136940E0024E96E000E01205D
:106AF000EA6EEECF04F0EECF05F015D024C403F01B
:106B00000F0E031603C000F0000E016E0036009059
:106B100001367D0E0024E96E000E0120EA6EEECFF4
:106B200004F0EECF05F004C0E9FF05C0EAFFEECFA8
:106B300001F001A403D00401010E286F15D020C478
:106B400001F01F0E01160150000AAFE020C401F051
:106B50001F0E01160150010AB3E020C401F01F0E00
:106B600001160150020AAFE0000166AF07D0280EFF
:106B7000636F040E646F6681020E676F1200000E71
:106B80000001685D02E1080E675D10E267C003F076
:106B900068C004F05F50000A03E1010E5F6E05D08B
:106BA0005F50010A02E1020E5F6E04D0080E036E10
:106BB000000E046E7DC0E1FF7EC0E2FFE6927DC064
:106BC000E1FF7EC0E2FFE6907DC0E9FF7EC0EAFF04
:106BD000EECF00F07DC0E1FF7EC0E2FF0450001068
:106BE000E66E010E7D25E16E000E7E21E26E03C091
:106BF000E6FF0350675D006E04506859016E00C0E7
:106C000067F001C068F0280E916F040E926F66B1B4
:106C10002FD0035004102BE063C0F6FF64C0F7FFD1
:106C200065C0F8FF0900F5CF00F091C0E1FF92C008
:106C3000E2FF00C0E6FF914B922B010E6325006E30
:106C4000000E6421016E000E6521026E00C063F02B
:106C500001C064F002C065F0010E035C006E000E1E
:106C60000458016E00C003F001C004F0D2D724D054
:106C70000350041021E063C0E9FF64C0EAFF91C043
:106C8000E1FF92C0E2FFEECFE6FF914B922B010EA7
:106C90006325006E000E6421016E00C063F001C028
:106CA00064F0010E035C006E000E0458016E00C01B
:106CB00003F001C004F0DCD7120004012251010AE4
:106CC00013E120C401F01F0E01160150000A0CE16F
:106CD0000001668F04012151030A04E1010E000145
:106CE000846F02D00001846B04012251000AD8A4F1
:106CF0008DD020C401F01F0E01160150020AD8A445
:106D000085D024C401F00F0E01160150000AD8B43A
:106D10007DD00001668F040124BF16D024C403F087
:106D20000F0E031603C000F0000E016E0036009037
:106D30000136940E0024E96E000E0120EA6EEECFBB
:106D400004F0EECF05F015D024C403F00F0E0316A7
:106D500003C000F0000E016E0036009001367D0E7B
:106D60000024E96E000E0120EA6EEECF04F0EECFB3
:106D700005F02151030A07E104C0E1FF05C0E2FF6D
:106D8000840EE66E43D024C400F00F0E0016700E81
:106D9000026E0F0E036E00500226D8B0032A02C006
:106DA000E9FF03C0EAFFFE0EEE14006EEECF01F025
:106DB000FF0E011602C0E1FF03C0E2FF00C0E6FFC4
:106DC00001C0E6FF24AF11D004C0E1FF05C0E2FF1F
:106DD000E66A040E0418006E00C004F004C0E1FF6F
:106DE00005C0E2FF400EE66E11D004C0E1FF05C011
:106DF000E2FF880EE66E040E0418006E00C004F078
:106E000004C0E1FF05C0E2FFC80EE66E12000401F7
:106E10002051800AD8A479D0C00E0001666F6AD0D4
:106E200000017F0E006E7F0E016E000E026E00C02C
:106E300063F001C064F002C065F0120E676F000ECF
:106E4000686F63D00001030E006E000E016E22C455
:106E500004F0000E056EFDDD810E0024E96E000ECB
:106E60000120EA6EEECF63F0EECF64F0EECF65F076
:106E7000020E6325F66E000E6421F76E000E65218A
:106E8000F86E0900F5CF00F00900F5CF01F000C061
:106E900067F001C068F039D0030E0401225D24E2DE
:106EA000030E006E000E016E22C404F0000E056E8B
:106EB000D0DD740E0024E96E000E0120EA6EEECFE4
:106EC00063F0EECF64F0EECF65F063C0F6FF64C010
:106ED000F7FF65C0F8FF0900F5CF00F000C067F0CC
:106EE000000E0001686F02D00001666B0ED0000139
:106EF000666B0BD004012351010A92E02351020A70
:106F0000A1E02351030AC8E0F2D712000001668F06
:106F1000710EB56F0F0EB66FB76B010EB86F000E26
:106F2000B96F3BDD8C0EB56F000EB66FB76B010EFF
:106F3000B86F000EB96F31DD22C48BF08B51000A9F
:106F400003E1100E5E6E0FD0200E5E6E010EB56F67
:106F5000000EB66F8B0EB76F000EB86F010EB96FD3
:106F6000000EBA6F34DD1200010E00016925E96ED2
:106F7000000E6A21EA6EEECF00F000C002F0000EB3
:106F80006F5D02E102506E5D03E26EC002F00AD056
:106F900002506E5D006E000E6F59016E00C06EF003
:106FA00001C06FF0036A0250035C1CE2280EE96E18
:106FB000040EEA6E0350E926D8B0EA2AEECF00F0BC
:106FC0006BC0E1FF6CC0E2FF00C0E6FF010E6B2565
:106FD000006E000E6C21016E00C06BF001C06CF001
:106FE000032AE1D7000E006E6F51005C02E16E5182
:106FF000000828E2010E6125E16E000E6221E26EBA
:10700000080EE66E020E6125E16E000E6221E26E50
:10701000280EE66E040EE66E69C0E9FF6AC0EAFF5C
:10702000EECF00F000BC07D061C0E1FF62C0E2FF1C
:10703000C80EE66E06D061C0E1FF62C0E2FF880EB6
:10704000E66E19D0010E6125E16E000E6221E26E3E
:10705000080EE66E020E6125E16E000E6221E26E00
:10706000200EE66E040EE66E61C0E1FF62C0E2FF34
:10707000840EE66E6D9F12000001606B7DC0E1FF23
:107080007EC0E2FFE66A040E7D19E16E7EC0E2FF7B
:10709000000EE21AE66A6DAF01D06D9F12006D9886
:1070A000000166BF49D06DAF28D0020E606F010E9F
:1070B0007D25E16E000E7E21E26EE66A7DC0E1FF75
:1070C0007EC0E2FFC80EE66E010E6125E16E000E85
:1070D0006221E26E080EE66E020E6125E16E000E80
:1070E0006221E26E280EE66E040EE66E61C0E1FFDC
:1070F00062C0E2FFC80EE66E1ED0010E6125E16E91
:10710000000E6221E26E080EE66E020E6125E16E4F
:10711000000E6221E26E200EE66E040EE66E61C085
:10712000E1FF62C0E2FF8C0EE66E7DC0E1FF7EC033
:10713000E2FF840EE66E82D06DBF80D0040120AFE6
:1071400055D0000168510401275D04E10001675139
:107150000401265D04E226C467F027C468F00FDD51
:10716000010E606F010E6125E16E000E6221E26E7C
:10717000080EE66E020E6125E16E000E6221E26EDF
:10718000200EE66E040EE66E61C0E1FF62C0E2FF13
:10719000800EE66E936B010E6925E16E000E6A218A
:1071A000E26E080EE66E020E6925E16E000E6A219F
:1071B000E26E200EE66E040EE66E69C0E1FF6AC064
:1071C000E2FF840EE66E010E936F020E7D25E16EE6
:1071D000000E7E21E26E280EE66E040EE66E7DC085
:1071E000E1FF7EC0E2FFC80EE66E28D00001020E6D
:1071F000606F010E7D25E16E000E7E21E26EE66A73
:107200007DC0E1FF7EC0E2FFC80EE66E010E612583
:10721000E16E000E6221E26E080EE66E020E61253E
:10722000E16E000E6221E26E280EE66E040EE66E3E
:1072300061C0E1FF62C0E2FFC80EE66E120020C42A
:1072400001F0600E0116050E006E005004E00132E0
:10725000019EFF0FFBD70150000A01E069D045D025
:107260000001668F080E5E6E63D0D1DD61D04EDE08
:107270005FD08B0E0001636F000E646F6681010E9C
:10728000676F668F55D00DDC53D017DD51D08C0E53
:10729000006E000E016E040124510026D8B0012AB0
:1072A00000C063F001C064F000016681010E676FE9
:1072B000668F3ED00001668F8C0EE16E000EE26E8E
:1072C00004012451E126D8B0E22A22C4E6FF30D0DE
:1072D000020E0001B56F000EB66FB76BB86BB96BDD
:1072E000BA6BE7EC34F024D023D004012151050A15
:1072F000B7E02151060AB9E02151090AB8E021514D
:10730000080AB7E02151000ABEE02151010ABDE0A0
:107310002151030ABAE021510A0AB9E021510B0AAE
:10732000C9E02151070AD4E021510C0ADDE0DCD785
:1073300012000001B151000A12E0B0C000F0000ECE
:10734000016E0036009001367D0E0024E96E000EBD
:107350000120EA6EEECF04F0EECF05F011D0B0C000
:1073600000F0000E016E003600900136940E0024ED
:10737000E96E000E0120EA6EEECF04F0EECF05F0CC
:10738000020E0424E16E000E0520E26EB2C0E6FF9C
:10739000B3C0E6FF010E0424E16E000E0520E26E8C
:1073A000B4C0E6FF04C0E9FF05C0EAFFEECF00F07D
:1073B00004C0E1FF05C0E2FF400E0014E66E04C009
:1073C000E9FF05C0EAFFEECF00F004C0E1FF05C011
:1073D000E2FF880E0010E66EB151000A1BE0B0C05B
:1073E00000F0000E016E0036009001367D0E002484
:1073F000026E000E0120036E02C0E9FF03C0EAFF27
:10740000040EEE18006E02C0E1FF03C0E2FF00C0F0
:10741000E6FF1AD0B0C000F0000E016E00360090FA
:107420000136940E0024026E000E0120036E02C08D
:10743000E9FF03C0EAFF040EEE18006E02C0E1FF90
:1074400003C0E2FF00C0E6FF04C000F005C001F089
:107450001200000E0001B11902E1000EB01902E1A4
:10746000016A09D0B0C0E9FFB1C0EAFFEECF00F079
:10747000016A00BE012A01C000F01200ED0E0001F9
:10748000816F7E0E826F000E836F980E746F7F0E79
:10749000756F000E766F3C0E776F7F0E786F000E63
:1074A000796F160E7A6F7F0E7B6F000E7C6F120065
:1074B000160E6F6E9F0E6B6E7B0E696E12007DC096
:1074C000E9FF7EC0EAFFEECF00F000AE05D07DC040
:1074D000E1FF7EC0E2FFE66A5F6A0001606B676BF6
:1074E000686B666BACDE030E0001B56F000EB66F05
:1074F000B76BB86BB96BBA6BE7EC34F0D0DD120048
:10750000200E5E5C03E36DB201D002D0006A33D07E
:1075100089C0B0F08AC0B1F09CDF00522BE1AFC04F
:10752000B0F0010EB16FACC0B2F0ADC0B3F0AEC000
:10753000B4F0FFDE00C089F001C08AF08D6B8E6B65
:107540008F6B906B89C0B0F08AC0B1F082DF0052BF
:1075500008E08D518E118F11901102E0006A0BD05E
:10756000F1D7010E8925E96E000E8A21EA6EEECF71
:1075700000F001D0006A12007DC0E9FF7EC0EAFF82
:10758000EECF00F0000E00BC010E0001AC6F040E47
:107590007D19006E00C07DF05E50080A0AE122C429
:1075A0006EFF6E50000803E2100E5E6E02D0040EF5
:1075B0005E6E6051010A2BE1020E7D25E16E000E28
:1075C0007E21E26E280E006E040E016E00C0E6FF02
:1075D00001C0E6FFBFEC35F05F50020A07E17DC055
:1075E000E1FF7EC0E2FF840EE66E10D0AC51000ACF
:1075F00007E17DC0E1FF7EC0E2FFC80EE66E06D067
:107600007DC0E1FF7EC0E2FF880EE66E01D034DD72
:10761000120000016051020A02E1A6DC1ED02CDD3E
:107620009351000A19E1010E6125E16E000E6221FD
:10763000E26E080EE66E020E6125E16E000E62211A
:10764000E26E200EE66E040EE66E61C0E1FF62C0DF
:10765000E2FF8C0EE66E01D0936B1200740E0001F7
:10766000B56F000EB66FB76BB86BB96BBA6BE7EC62
:1076700034F06D92699468A403D0FB0E6816FBD7B2
:107680001200FD0E00018515016E026AFF0E021642
:10769000000E021802E1000E01186BE17E0E851546
:1076A000016E01C003F00332039E03C000F0000E20
:1076B000016E003600900136003600900136000E53
:1076C0000024026E040E0120036E02C069F003C0A4
:1076D0006AF002C061F003C062F0040E6119006E2E
:1076E00000C061F002C0E9FF03C0EAFFEECF00F086
:1076F00000C001F03C0E01160132019E0132019ED4
:1077000001500D0A34E1020E6925E96E000E6A216E
:10771000EA6EEECF01F0EECF02F00250040A02E171
:10772000280E011822E1020E6925E16E000E6A2181
:10773000E26E200EE66E040EE66EA66B080EA65DE7
:1077400014E2200EE16E040EE26EA651E126D8B0DE
:10775000E22A280EE96E040EEA6EA651E926D8B098
:10776000EA2AEECFE6FFA62BE9D7A9DE01D051DF4A
:107770000DD0FD0E8515016E026AFF0E0216000E79
:10778000021802E1040E011801E1F6DE1200A6C0A3
:1077900002F0A7C003F0A9C000F0AAC001F0010EDA
:1077A0000001A95F000EAA5B0050011009E002C0B1
:1077B000E1FF03C0E2FFA8C0E6FF024A032AEBD7BD
:1077C0001200D08EA28AA08AF28E120070A019D068
:1077D00069C0E9FF6AC0EAFFEECF01F00150800AFC
:1077E0000FE17DC0E9FF7EC0EAFFEECF01F001505E
:1077F000840A06E169C0E1FF6AC0E2FF8C0EE66E12
:107800007090DF0E68161200A19A12006984EF0EC4
:1078100068166D82750E0001B56F000EB66FB76BFE
:10782000B86BB96BBA6BE7EC34F0120027DE986BDB
:10783000996B896B8A6B6A6A686A3ADE6D8C6E6ACC
:10784000710EB56F0F0EB66FB76B010EB86F000EED
:10785000B96FCDEC34F06D9CA66B080EA65D16E2F8
:10786000A6C000F0000E016E003600900136003612
:1078700000900136000E0024E16E040E0120E26E3D
:10788000E66AE66AE66AE66AA62BE7D7160E706E27
:1078900068A603D0F70E6816FBD7666B6D6B6E6B30
:1078A0006F6B6D98080E7D6F040E7E6F8B6B5E6A3A
:1078B0001200A6C0ACF0A7C0ADF0A8C0AEF0010E9B
:1078C0000001AF6F1DDE1200200E5E5C03E36DB29F
:1078D00001D002D0006A23D098C0B0F099C0B1F0B6
:1078E000B8DD00521BE1010E9825E96E000E9921CA
:1078F000EA6EEECF00F000C0AAF0A9C0B0F0B16B04
:10790000A6C0B2F0A7C0B3F0A8C0B4F012DD00C0AA
:1079100098F001C099F0AAC000F001D0006A1200EE
:10792000F2CF02F0F29EA6C0F6FFA7C0F7FFA8C0F4
:10793000F8FFAAC0E9FFABC0EAFF0A00016A200E07
:10794000015C07E2EECFF5FF00000F000000012A06
:10795000F6D7A68EBF0EA616A684550EA76EAA0E43
:10796000A76EA682A69402BE02D0F29E01D0F28E2D
:1079700012005E50000A0AE16D6A696A99DD21DF32
:107980006DB602D06D86FCD7010E5E6E12005E50A1
:10799000000A09E16D6A696A8BDD6DB602D06D86F9
:1079A000FCD7010E5E6E5E50010A08E16DBA06D08A
:1079B000686A696A69806988020E5E6E68A405D08B
:1079C00069A403D0FB0E681649DE6DA202D01CDF4D
:1079D00077D068A018D069A016D028DF040E5E6E9C
:1079E000200E0401026F040E036F080E016F000EDB
:1079F0000015006E00C000F48C0E0011006E00C077
:107A000000F4FE0E681668A805D069A803D0FEDE53
:107A1000EF0E681668AC11D069AC0FD0730E000180
:107A2000B56F000EB66FB76BB86B010EB96F000E75
:107A3000BA6FE7EC34F0BF0E681668AA03D069AAE3
:107A400001D0C4DE68A210D069A20ED0FF0E0001E2
:107A5000B56F3F0EB66FB76BB86B010EB96F000E06
:107A6000BA6FE7EC34F06A6A040E5E5C02E2CCDEC8
:107A700027D069A624D00001A26B040EA25D1FE2EC
:107A800068A619D06CCF85F0F70E6816780E8515AC
:107A9000016E0150000A02E1F4DD0CD0720EB56FE8
:107AA000000EB66F850EB76F000EB86FB96BBA6B6C
:107AB000E7EC34F001D003D00001A22BDED7A4DE26
:107AC00012000F0E0501406FA2C041F5400E0001EB
:107AD000A66F050EA76F400EA86FEBDE12001550C3
:107AE000000A17E1000E000A03E10F0E050100195C
:107AF00001E00FD001C515F002C518F003C519F05B
:107B000004C51AF005C51BF006C516F007C517F029
:107B100000D012009AC0A6F09BC0A7F0400E000152
:107B2000A86F010EA96FD0DE1200100E0C6E940E1D
:107B30000D6E0D2EFED70C2EFCD700001200400E4D
:107B4000E16E050EE26E2B0E016EC20EF66E7E0E1B
:107B5000F76E000EF86E0900F5CF00F000C0E6FFEA
:107B60000106F9E1400E0001A66F050EA76F400E59
:107B7000A86F9FDE12009C0E0C6ED70E0D6E0D2EA0
:107B8000FED70C2EFCD712001C0E5C5C0001A26F0D
:107B9000000E5D58A36F1C0E5C6E000E5D6E800EB5
:107BA000006E800EA319005C02E1A251000823E2DE
:107BB00018C0A6F019C0A7F01AC0A8F01BC0A9F001
:107BC0005CC0AAF05DC0ABF0ABDE200E0001A25F8E
:107BD000000EA35B200E5C24006E000E5D20016E83
:107BE00000C05CF001C05DF0200E1826000E1922C6
:107BF0001A221B22D4D712006D6A696A5E6A1200CB
:107C00003DDC986B996B896B8A6B6A6A686A50DC99
:107C10006D8C6E6A710EA66F0F0EA76FA86B010EAA
:107C2000A96F000EAA6FB3DD6D9CA26B080EA25D5A
:107C300016E2A2C000F0000E016E00360090013680
:107C4000003600900136000E0024E16E040E012083
:107C5000E26EE66AE66AE66AE66AA22BE7D7160EE5
:107C6000706E68A603D0F70E6816FBD7666B6D6B57
:107C70006E6B6F6B6D98080E7D6F040E7E6F8B6B55
:107C80005E6A1200F2CF00F0F29EA2C0F6FFA3C01F
:107C9000F7FFA4C0F8FFA68EBF0EA616A684A6887E
:107CA000550EA76EAA0EA76EA682A69400BE02D09D
:107CB000F29E01D0F28E1200000E046E050E056ECB
:107CC000036A1650171003E1010E006E30D01C0E2F
:107CD0005C5C016E000E5D58026E000E021802E13F
:107CE000400E011803E1010E006E21D00350400A3E
:107CF00002E1006A1CD004C0E9FF05C0EAFF5CC0D5
:107D0000E1FF5DC0E2FFEECFE6FF010E5C24006EF6
:107D1000000E5D20016E00C05CF001C05DF0044A01
:107D2000052A010E165E000E175A032ACAD7120042
:107D300063DF1200000E006E040E016E0050011091
:107D400000E01200010E0001866F9EC09AF09FC0F5
:107D50009BF0A0C087F0A1C088F052DF000E016E3A
:107D60000150010A01E105DE12000900F5CFE6FF2E
:107D70000006FBE10106F9E11200880E00019E6F8A
:107D8000130E9F6F04DEC6DE005213E0A8DE0BD098
:107D900015C0A2F096DE156AEEDE010E006E19D057
:107DA000CEDE156A06D01550030AF2E01550020A1D
:107DB000F7E0BBDE9EC000F09FC001F0010E0001A5
:107DC0009E5F000E9F5B0050011002E1006A01D02F
:107DD000D9D7120000019E6B1C0E5C6E000E5D6E0A
:107DE000D6DD98DE0052D8B46AD079DE5CD00001CE
:107DF0009E5321E061DF00521DE0000E1B5C08E194
:107E0000000E1A5C05E1650E195C02E1400E185C7B
:107E100001E2BADE15C0A2F054DE1C0E5C6E000E4C
:107E20005D6E000E171802E1000E161803E1000146
:107E30009E6B156A03D00001010E9E6F40D016C0E4
:107E400000F017C001F0010E165E000E175A005028
:107E500001101CE0000E1B5C08E1000E1A5C05E13D
:107E6000650E195C02E1400E185C09E218C0A2F030
:107E700019C0A3F01AC0A4F01BC0A5F003DF400E88
:107E8000185E000E195A1A5A1B5AD9D715C0A2F0FB
:107E900018DE156A14D015C0A2F013DE156A0FD0D3
:107EA000FF00156A0CD015500B0AA1E01550150AF9
:107EB000C6E01550010AEFE01550040AF1E090D732
:107EC00012002B0102080080000003400004200083
:107ED0000500130640650000075374617274555322
:107EE000420000000000000000000000000902291C
:107EF00000010100803209040000020300000009B3
:107F00002101010001222100070581034000010732
:107F100005010340000126035500530042002000E4
:107F2000480049004400200042006F006F007400C8
:107F30006C006F00610064006500720022034D0058
:107F400069006B0072006F0065006C0065006B00DB
:107F5000740072006F006E0069006B006100060023
:107F6000FF0901A10119012940150026FF0075082C
:107F70009540810219012940750895409102C0126F
:107F8000010002000000083412010001000102009B
:107F900001000000000000000403090410EE15F0C9
:107FA000070E006E010E016E910EF66E7F0EF76EDB
:107FB000000EF86EB5EC3EF01200FFFFFFFFFFFF72
:107FC000FFFFFFFFFFFFFFFFFFFFFFFFFFFFFFFFC1
:107FD000FFFFFFFFFFFFFFFFFFFFFFFFFFFFFFFFB1
:107FE000FFFFFFFFFFFFFFFFFFFFFFFFFFFFFFFFA1
:107FF000FFFFFFFFFFFFFFFFFFFFFFFFFFFFFFFF91
:020000040020DA
:08000000FFFFFFFFFFFFFFFF00
:020000040030CA
:0E000000214E2E1E008181000FC00FE00F4028
:0200000400F00A
:10000000FFFFFFFFFFFFFFFFFFFFFFFFFFFFFFFF00
:10001000FFFFFFFFFFFFFFFFFFFFFFFFFFFFFFFFF0
:10002000FFFFFFFFFFFFFFFFFFFFFFFFFFFFFFFFE0
:10003000FFFFFFFFFFFFFFFFFFFFFFFFFFFFFFFFD0
:10004000FFFFFFFFFFFFFFFFFFFFFFFFFFFFFFFFC0
:10005000FFFFFFFFFFFFFFFFFFFFFFFFFFFFFFFFB0
:10006000FFFFFFFFFFFFFFFFFFFFFFFFFFFFFFFFA0
:10007000FFFFFFFFFFFFFFFFFFFFFFFFFFFFFFFF90
:10008000FFFFFFFFFFFFFFFFFFFFFFFFFFFFFFFF80
:10009000FFFFFFFFFFFFFFFFFFFFFFFFFFFFFFFF70
:1000A000FFFFFFFFFFFFFFFFFFFFFFFFFFFFFFFF60
:1000B000FFFFFFFFFFFFFFFFFFFFFFFFFFFFFFFF50
:1000C000FFFFFFFFFFFFFFFFFFFFFFFFFFFFFFFF40
:1000D000FFFFFFFFFFFFFFFFFFFFFFFFFFFFFFFF30
:1000E000FFFFFFFFFFFFFFFFFFFFFFFFFFFFFFFF20
:1000F000FFFFFFFFFFFFFFFFFFFFFFFFFFFFFFFF10
:00000001FF
